:100000000C940E020C9436020C9436020C943602B8
:100010000C9436020C9436020C9436020C94360280
:100020000C9436020C9436020C9436020C94360270
:100030000C9436020C9436020C9436020C94360260
:100040000C94CE330C9436020C949F050C94DB0573
:100050000C9436020C9436020C9436020C94360240
:100060000C9436020C9436028108810887088A08AD
:100070008D0890089308960899089C089F08A20884
:10008000A508A808AB08AE08B108084AD73B3BCE84
:10009000016E84BCBFFDC12F3D6C74319ABD568387
:1000A0003DDA3D00C77F11BED9E4BB4C3E916BAA3F
:1000B000AABE000000803F05A84CCDB2D44EB9388E
:1000C00036A9020C50B9918688083CA6AAAA2ABE75
:1000D000000000803F0664EC1B3C04BC163E3BE580
:1000E000B93CC93C37C29E5A3D660498083EEA694D
:1000F000AAAA3E000000803FEAEB00EAEC00426F53
:100100006F74696E672075703AEDF2F2F2F2F2F2F6
:10011000F2F30057616974696E6720666F727C4DF7
:1001200041564C696E6B20686561727462656174DA
:10013000732E2E2E00C820202020202020202020BA
:100140002020C900C820202020202020202020207E
:1001500020C97C00D8202020202020202020202002
:1001600020D97C00C82020202020202020202020F2
:1001700020C97C00C82020202020202020202020F2
:1001800020C97C00050304057C1513141500426189
:100190007474657279207761726E696E67200020D1
:1001A00020205374616C6C2053706565642020209E
:1001B00000202020204F76657273706565642020D2
:1001C0002020001820209091200020202020202096
:1001D000BABBBCBDBE7C202020202020CACBCCCD09
:1001E000CE7C4172647543414D204F53442076329A
:1001F0002E32004368617220446F6E650A005265BA
:1002000061647920666F7220466F6E740A005570C3
:1002100064617465204368617253657400EEEEEEAC
:10022000EEEEEEEEEE00EEEEEEEEEEEEEE00EEEECA
:10023000EEEEEEEEF000EEEEEEEEEEF0F200EEEEB2
:10024000EEEEF0F2F200EEEEEEF0F2F2F200EEEE92
:10025000F0F2F2F2F200EEF0F2F2F2F2F200EFF26D
:10026000F2F2F2F2F200F1F2F2F2F2F2F200526580
:100270007175657374696E6720446174615374723B
:1002800065616D732E2E2E00454550524F4D206DE9
:10029000617070696E67206F757464617465642144
:1002A0007C55706461746520776974682074686532
:1002B000204F534420546F6F6C2E0000407A10F38F
:1002C0005A00A0724E18090010A5D4E80000E87684
:1002D00048170000E40B54020000CA9A3B000000DB
:1002E000E1F505000080969800000040420F0000F4
:1002F00000A08601000000102700000000E80300B5
:100300000000006400000000000A0000000000017E
:1003100000000000002C76D888DC674F0823DFC17E
:10032000DFAE59E1B1B796E5E3E453C63AE6519939
:100330007696E8E6C28426EB898C9B62ED407C6F62
:10034000FCEFBC9C9F40F2BAA56FA5F490055A2A19
:10035000F75C936B6CF9676DC11BFCE0E40D47FE25
:10036000F520E6B500D0ED902E030094357705001A
:1003700080841E080000204E0A000000C80C3333A1
:1003800033330F986E12831141EF8D2114893BE6B0
:100390005516CFFEE6DB18D1844B381BF77C1D9039
:1003A0001DA4BBE424203284725E228100C9F124A2
:1003B000ECA1E53D276E616E00696E6600000000ED
:1003C00000240027002A0000000000250028002B40
:1003D0000000000000230026002900040404040497
:1003E00004040402020202020203030303030301E2
:1003F00002040810204080010204081020010204B9
:10040000081020000000070002010000030406009D
:1004100000000000000000001F072F2B11241FBE4A
:10042000CFEFD8E0DEBFCDBF14E0A0E0B1E0E8E759
:10043000F3E702C005900D92A836B107D9F716E090
:10044000A8E6B4E001C01D92A838B107E1F714E0B6
:10045000CCE1D4E004C02297FE010E94B639C83135
:10046000D107C9F70E9455350C94BA390C94000095
:10047000283008F027E03327DA01990F311D87FD76
:10048000916000966105710539F432602E5F3D93ED
:1004900030E32A95E1F708959F3F30F080387105E9
:1004A000610509F03C5F3C5F3D93913008F0806846
:1004B000911DDF93CF931F930F93FF92EF92192F0C
:1004C000987F9695E92F96959695E90FFF27EB5E15
:1004D000FC4F99273327EE24FF24A701E70105905D
:1004E0000894079428F4360FE71EF81E491F511D83
:1004F000660F771F881F991F0694A1F70590079430
:1005000028F4E70EF81E491F561FC11D770F881FDC
:10051000991F661F0694A1F70590079428F4F80E1A
:10052000491F561FC71FD11D880F991F661F771FB0
:100530000694A1F70590079420F4490F561FC71F92
:10054000D81F990F661F771F881F0694A9F78491FB
:100550001095177041F0D695C79557954795F79424
:10056000E7941A95C1F7EBEBF2E0689415901591BA
:1005700035916591959105907FE27395E118F10AA7
:10058000430B560BC90BD009C0F7E10CF11E431FFA
:10059000561FC91FD01D7EF4703311F48A95E6CF23
:1005A000E894015030F0080F0AF40027021708F40D
:1005B000202F2395022F7A3328F079E37D932A9513
:1005C000E9F710C07D932A9589F60694979567956B
:1005D000379517951794E118F10A430B560BC90B81
:1005E000D00998F023957E9173957A3308F070E3E3
:1005F0007C932013B8F77E9170617D9330F08395E2
:1006000071E37D9370E32A95E1F71124EF90FF9059
:100610000F911F91CF91DF91992787FD90950895B4
:10062000FA01AA27283051F1203181F1E8946F9323
:100630006E7F6E5F7F4F8F4F9F4FAF4FB1E03ED0C9
:10064000B4E03CD0670F781F891F9A1FA11D680F67
:10065000791F8A1F911DA11D6A0F711D811D911D9A
:10066000A11D20D009F468943F912AE0269F11240F
:100670003019305D3193DEF6CF010895462F477073
:10068000405D4193B3E00FD0C9F7F6CF462F4F70CE
:10069000405D4A3318F0495D31FD4052419302D02C
:1006A000A9F7EACFB4E0A6959795879577956795D2
:1006B000BA95C9F700976105710508959B01AC01D2
:1006C0000A2E06945795479537952795BA95C9F7F9
:1006D000620F731F841F951FA01D0895FC010590D4
:1006E000615070400110D8F7809590958E0F9F1F34
:1006F0000895FC016150704001900110D8F7809579
:1007000090958E0F9F1F0895FC011382128288EE30
:1007100093E0A0E0B0E084839583A683B7838CE068
:1007200093E0918380830895FC018089803419F4DB
:1007300021E030E002C020E030E0C9010895FC0172
:10074000818990E00895FC01648745876687478723
:10075000089580E090E0089580E090E0089580E0C2
:1007600090E008950895EF92FF921F93CF93DF9347
:10077000162F7A0186E060E00E94013584E696E05B
:1007800060E00E94132B84E696E060E00E94132B49
:1007900084E696E069E00E94132B84E696E0612FE0
:1007A0000E94132BC0E0D0E0F701EC0FFD1F108179
:1007B00084E696E06AE00E94132B84E696E06C2FB4
:1007C0000E94132B84E696E06BE00E94132B84E6D4
:1007D00096E0612F0E94132B2196C633D10521F795
:1007E00084E696E068E00E94132B84E696E060EAD7
:1007F0000E94132B84E696E060EA0E94132B85FD8D
:10080000F9CF84E696E060E00E94132B84E696E040
:100810006CE00E94132B86E061E00E940135DF91BD
:10082000CF911F91FF90EF9008951F93CF93DF9387
:10083000EC01162F86E060E00E94013584E696E028
:1008400060E00E94132B112319F0113059F404C0F9
:1008500084E696E0688904C068896C6184E696E065
:100860000E94132B86E061E00E940135DF91CF9159
:100870001F910895EF92FF920F931F938EE1489F6F
:1008800070011124E60EF11C86E060E00E94013543
:1008900004E616E0C80165E00E94132BC8016F2D25
:1008A0000E94132BC80166E00E94132BC8016E2D15
:1008B0000E94132B1F910F91FF90EF900895EF92DC
:1008C000FF920F931F937C0104E616E0C80167E0D6
:1008D0000E94132BC8016FEF0E94132B86E061E08A
:1008E0000E940135F70187858F5F87871F910F91E0
:1008F000FF90EF900895EF92FF920F931F93FC01EA
:10090000E7848EE1E89E700111248685E80EF11CD3
:1009100086E060E00E94013504E616E0C80164E06C
:100920000E94132BC80163E00E94132BC80165E0ED
:100930000E94132BC8016F2D0E94132BC80166E083
:100940000E94132BC8016E2D0E94132B1F910F9133
:10095000FF90EF9008951F93CF93DF93EC01162F34
:100960006C3731F40E945F04CE010E947B040AC000
:1009700084E696E067E00E94132B84E696E0612F00
:100980000E94132B81E090E0DF91CF911F91089599
:100990000F931F9386E060E00E94013504E616E0A5
:1009A000C80164E00E94132BC80164E00E94132B6D
:1009B00086E061E00E9401351F910F9108951F9319
:1009C000CF93DF93EC01188A16E0198B86E796E047
:1009D00060E973E00E94F931813049F480E4888B4A
:1009E00088E0898B86E060E00E94013502C0188AA9
:1009F000198B86E060E00E940135DF91CF911F9155
:100A000008951F93CF93DF93EC0186E061E00E948D
:100A1000C23482E060E00E94C23482E061E00E9461
:100A20000135CE010E94DF0486E060E00E940135BE
:100A300084E696E06CEE0E94132B84E696E06FEF5E
:100A40000E94132B182F84E696E060E00E94132B7F
:100A50006889626084E696E00E94132B62E370E08E
:100A600080E090E00E94243484E696E06CE60E94E8
:100A7000132B1F7E84E696E0612F0E94132B1092A9
:100A800069041092680417C0609168047091690449
:100A9000605F84E696E00E94132B84E696E060E0B7
:100AA0000E94132B809168049091690401969093A1
:100AB00069048093680480916804909169040C979C
:100AC0001CF3CE0161E00E941504DF91CF911F91CC
:100AD0000895CF92DF92EF92FF920F931F93CF93DF
:100AE000DF938C016B017A01C0E0D0E01CC0F601FD
:100AF000EC0FFD1F60810115110521F0013011057A
:100B000089F405C0E0917706F091780604C0E09181
:100B10007906F0917A06A081B1812D913C91CF01A7
:100B2000F90109952196CE15DF0508F3DF91CF91E4
:100B30001F910F91FF90EF90DF90CF9008951F923B
:100B40000F920FB60F9211242F933F934F938F93D1
:100B50009F93EF93FF934091C600209165063091DB
:100B600066062F5F3F4F8091690690916A062823A1
:100B7000392380916706909168062817390779F024
:100B80008091650690916606E0916B06F0916C0687
:100B9000E80FF91F40833093660620936506FF91A6
:100BA000EF919F918F914F913F912F910F900FBE99
:100BB0000F901F9018951F920F920FB60F9211244D
:100BC0002F933F938F939F93EF93FF9320916F0603
:100BD0003091700680916D0690916E062817390746
:100BE000E9F080916F0690917006E0917306F091A4
:100BF0007406E80FF91F80818093C60080916F060C
:100C000090917006019620917106309172068223B0
:100C100093239093700680936F0610C020916D0609
:100C200030916E0680916F069091700628173907F3
:100C300029F48091C1008F7D8093C100FF91EF91D5
:100C40009F918F913F912F910F900FBE0F901F900A
:100C500018952F923F924F925F926F927F928F9250
:100C60009F92AF92BF92CF92DF92EF92FF920F933B
:100C70001F93DF93CF93CDB7DEB72E970FB6F894BF
:100C8000DEBF0FBECDBF06E214E06AE1E62E64E0EF
:100C9000F62E53E0C52ED12CCC0EDD1E42E4242EC0
:100CA0003AE0432E512C4C0E5D1E2FE0622E712C2B
:100CB0006C0E7D1E99E0892E912C8C0E9D1E84E970
:100CC000382E5E010894A11CB11C2091CD053091F5
:100CD000CE05F8014081F701808191819C838B834F
:100CE0002D833E834F83F1E0F8878EEF898796E06E
:100CF0009A87909152069B878091FC028C87809105
:100D0000FD028D872E869F5F909352066FEF7FEFD7
:100D1000F2011CC021912627822F8295807F822795
:100D200090E0382F2227AC01A3E0440F551FAA956D
:100D3000E1F724273527672F772762277327A4E059
:100D400095958795AA95E1F768277927E615F70520
:100D500009F7F6011AC081918627282F2295207F56
:100D6000282730E0722F6627C90143E0880F991FBA
:100D70004A95E1F7682779276A277B27B4E03595FC
:100D80002795BA95E1F762277327A72FBB27E815A8
:100D9000F90509F7862F8325282F2295207F2827FC
:100DA00030E0922F8827A90163E0440F551F6A9510
:100DB000E1F7842795278A279B2744E035952795D7
:100DC0004A95E1F78227932789839A8380E090E010
:100DD000BF0146E050E00E94690580E090E0B60166
:100DE00046E050E00E94690580E090E0B50142E0F5
:100DF00050E00E9469050F5F1F4FE2E0F0E0EE0E49
:100E0000FF1EF4E00C321F0709F05FCF2E960FB6DD
:100E1000F894DEBF0FBECDBFCF91DF911F910F9130
:100E2000FF90EF90DF90CF90BF90AF909F908F900A
:100E30007F906F905F904F903F902F9008958F928A
:100E4000AF92CF92EF92FF920F931F938EEE94E0AA
:100E500060E045EC50E024EC30E000EC10E0F1EC18
:100E6000EF2EF12CCC24C394E8E9AE2E70E2872E4D
:100E70000E94692B8BE095E00E94840310921E056E
:100E800010921F0510922005109221051092220544
:100E90001092230510922405109225051092270523
:100EA0001092260510921D051F910F91FF90EF9053
:100EB000CF90AF908F90089586E796E06AE773E051
:100EC0000E94F9318823E9F486E696E6A6E6B0E4C6
:100ED0008093280590932905A0932A05B0932B05AC
:100EE00080E090E0A0E8BFE380932C0590932D056F
:100EF000A0932E05B0932F0581E8809330058DE8EF
:100F00001CC082E598EBAEE0B0E480932805909396
:100F10002905A0932A05B0932B0585E89BEEA1E552
:100F2000B0E480932C0590932D05A0932E05B093EB
:100F30002F058BEF8093300586E680933105089569
:100F4000CF93DF9386E796E06CE773E00E94F93178
:100F50008093730586E796E06EE773E00E94F931AF
:100F60008093720586E796E060E873E00E94F931AD
:100F70008093740586E796E06EE873E00E94F9318D
:100F80008093AB0586E796E06AE873E00E94F9314A
:100F90008093A20586E796E064E873E00E94F93149
:100FA0008093C50586E796E066E873E00E94F93114
:100FB0008093C40586E796E06CE873E00E94F931FF
:100FC00010927705882319F081E08093770586E7F2
:100FD00096E062E973E00E94F9318093750586E737
:100FE00096E064E973E00E94F93180937605C0E0F1
:100FF000D0E0BE0168567C4F86E796E00E94F9314A
:10100000FE01E654FA4F8083882321F02196C830F0
:10101000D10579F7C654DA4F1982DF91CF9108953F
:10102000BC0186E796E00E94F93108951F93282FAE
:10103000362F142F8BE095E0622F432F0E943A0445
:101040001530F9F0163060F41230A9F0133018F4AE
:10105000113001F50EC0133081F01430D9F40FC0F7
:10106000173099F0173078F0183089F0193091F472
:1010700010C026E00FC027E00DC028E00BC029E01B
:1010800009C02AE007C02BE005C02CE003C02DE01A
:1010900001C02EE000D000D000D0EDB7FEB73196F1
:1010A0008BE095E0ADB7BEB712969C938E931197E7
:1010B00080E091E093838283822F992787FD90952A
:1010C000958384830E94482B8DB79EB706960FB6F2
:1010D000F8949EBF0FBE8DBF1F910895EF92FF92AF
:1010E0000F931F93CF93DF93E82FF0E0E131F105E9
:1010F00058F4EC5CFF4FEE0FFF1F0590F491E02DCC
:10110000099490E981E92FC090E080E02CC092E939
:1011100083E929C094E985E926C096E987E923C0D7
:1011200098E989E920C09AE98BE91DC09CE98DE91D
:101130001AC09EE98FE917C090EA81EA14C092EACA
:1011400083EA11C094EA85EA0EC096EA87EA0BC0EA
:1011500098EA89EA08C09AEA8BEA05C09CEA8DEA17
:1011600002C09EEA8FEA2BE035E0C92FDD27C7FDDC
:10117000D095E82EFF24E7FCF094613009F04AC0D6
:101180008DB79EB740970FB6F8949EBF0FBE8DBF28
:101190000DB71EB70F5F1F4FADB7BEB712963C938A
:1011A0002E93119783E091E0F801938382838CEF73
:1011B00090E095838483609134057091350580912A
:1011C00036059091370520912805309129054091E9
:1011D0002A0550912B050E942A38D80116966D9346
:1011E0007D938D939C931997809130051A968C93DB
:1011F0001A971B961C921B971D96DC93CE931C97F7
:101200001F96FC92EE921E970E94482BEDB7FEB7F8
:1012100070961EC08DB79EB708970FB6F8949EBF04
:101220000FBE8DBFEDB7FEB73196ADB7BEB7129604
:101230003C932E93119782E191E093838283D5832F
:10124000C483F782E6820E94482BEDB7FEB738963A
:101250000FB6F894FEBF0FBEEDBFDF91CF911F9187
:101260000F91FF90EF9008952F923F924F925F92CF
:101270006F927F928F929F92AF92BF92CF92DF92A6
:10128000EF92FF920F931F93DF93CF93CDB7DEB70B
:101290006C970FB6F894DEBF0FBECDBF8B8F6C8FEF
:1012A00080913205682F772767FD70959B0177FF46
:1012B00004C022273327261B370B2A35310589F432
:1012C0008AE590E00E945039882777FD8095982F15
:1012D0000E94F73621EE3AEF43EB52E40E942A389F
:1012E00008C0682F772767FD7095872F972F0E947A
:1012F000F73625E33AEF4EE85CEB0E942A38962E4B
:10130000E72E8C0180913305682F772767FD709554
:101310009B0177FF04C022273327261B370B2A3572
:10132000310589F48AE590E00E945039882777FDDD
:101330008095982F0E94F73621EE3AEF43EB52E466
:101340000E942A3808C0682F772767FD7095872F7D
:10135000972F0E94F73625E33AEF4EE85CE30E94B0
:101360002A385B016C01292D3E2DB901C8010E946C
:10137000FE3820E030E044E352E40E942A380E9424
:101380008D380E94C4367B018C01B501C6010E94D4
:10139000FE381B012C015E010894A11CB11CBA8E01
:1013A000A98E1EEBC12E1FEFD12E3701882477FCAA
:1013B0008094982CB601882777FD8095982F0E94FD
:1013C000F7369B01AC01C201B1010E942A387B01B2
:1013D0008C01C401B3010E94F7369B01AC01C80126
:1013E000B7010E948F3520E030E044E352E40E94D0
:1013F0008F3520E030E040E85FE30E948E350E94A8
:10140000C436E98DFA8D61937193FA8FE98F4CE0C0
:1014100050E0C40ED51E5EE4C516D10459F6EB8C1F
:10142000BEEE8B2EBFEF9B2EA9E1CA2ED12CCC0E87
:10143000DD1EF50120813181C901019789359105B2
:1014400068F56EEE7FEF0E9450398B010B5F1F4FE6
:101450002B553040089DC001099D900D189D900DA1
:101460001124A901481B590BCA0162E070E00E94D7
:101470005039882777FD8095982F0E94F7360E9473
:101480008D380E94C436AB01672B11F441E050E067
:101490006C8D600F61508E2D0E94160882E090E0E6
:1014A000A80EB91EE394AC14BD0419F66C960FB6E1
:1014B000F894DEBF0FBECDBFCF91DF911F910F918A
:1014C000FF90EF90DF90CF90BF90AF909F908F9064
:1014D0007F906F905F904F903F902F900895609114
:1014E000400570914105809142059091430520E0AF
:1014F00030E040E152E40E942A3820E030E044EB42
:1015000053E40E945C360E948D380E94C4369B01D1
:101510002550304037FF03C09B01215E3F4FA6E4BA
:10152000B5E0F901E45DFB4F80818C932F5F3F4F65
:101530002432310514F020E030E0119685E0A13529
:10154000B80779F71C9208950F931F93282F462F01
:101550008BE095E0622F0E94A3038BE095E00E9450
:101560007B0427E131E080913805823009F041C0E9
:1015700080913905882309F44DC0813009F454C0A5
:10158000823019F422E231E07EC0833009F465C074
:10159000843009F471C0853009F469C0863009F4DB
:1015A00061C0873091F1883019F420E431E06BC0DC
:1015B000893019F425E431E066C08A3019F42AE450
:1015C00031E061C08B3019F42FE431E05CC08D3024
:1015D00019F424E531E057C08E3019F429E531E0E3
:1015E00052C08F30A9F1803109F04DC023E631E0BF
:1015F0004AC0813009F047C080913905882319F429
:1016000028E631E040C0813019F42BE331E03BC0E3
:10161000823019F428E131E036C0833019F42DE628
:1016200031E031C0843019F42DE131E02CC0853037
:1016300019F422E731E027C0863019F427E731E0BA
:1016400022C0873019F42CE731E01DC0883019F42E
:101650002EE531E018C08A3019F427E231E013C0DA
:101660008B3019F426E331E00EC08C3019F421E3FD
:1016700031E009C08F3019F42CE231E004C0803130
:1016800011F421E831E08DB79EB708970FB6F894B2
:101690009EBF0FBE8DBFEDB7FEB731960BE015E0D4
:1016A000ADB7BEB712961C930E93119786E891E0E2
:1016B0009383828380EE90E09583848337832683AF
:1016C0000E94482B8DB79EB708960FB6F8949EBF20
:1016D0000FBE8DBFC8010E945F041F910F91089536
:1016E0000F931F93282F462F0BE015E0C801622FA0
:1016F0000E94A303C8010E947B0480913A0560E028
:101700000E946E08C8010E945F041F910F91089506
:10171000EF92FF920F931F93282F462F0BE0E02E9E
:1017200005E0F02EC701622F0E94A303C7010E94AB
:101730007B048DB79EB740970FB6F8949EBF0FBE3F
:101740008DBF0DB71EB70F5F1F4FEDB7FEB7F2820B
:10175000E1828BE891E0F8019383828387E590E052
:101760009583848380913B0586831782118610863A
:1017700060913C0570913D0580E090E00E94F53657
:1017800020912C0530912D0540912E0550912F056B
:101790000E942A38F8016287738784879587809131
:1017A0003105868717860E94482B8DB79EB74096D5
:1017B0000FB6F8949EBF0FBE8DBFC7010E945F0495
:1017C0001F910F91FF90EF900895282F462F8BE0E7
:1017D00095E0622F0E94A3038BE095E00E947B04BA
:1017E00060913E0570913F05882777FD8095982F81
:1017F0000E94F73620914005309141054091420505
:10180000509143050E948E3520E030E044EB53E4D4
:101810000E945C3620E030E040E851E40E942A3823
:101820000E948D3820E030E040E85FE30E948F3571
:101830000E94C436862F6093440567FF03C0805F13
:10184000809344058091440560E00E946E088BE01F
:1018500095E00E945F0408950F931F93282F462F51
:101860000BE015E0C801622F0E94A303C8010E948B
:101870007B048DB79EB70C970FB6F8949EBF0FBE32
:101880008DBFEDB7FEB73196ADB7BEB712961C93BC
:101890000E9311978AE991E09383828384EA91E021
:1018A0009583848380ED90E09783868386E495E03A
:1018B0009187808781ED90E0938782870E94482BF3
:1018C0008DB79EB70C960FB6F8949EBF0FBE8DBF16
:1018D000C8010E945F041F910F9108950F931F93F9
:1018E000282F462F0BE015E0C801622F0E94A303AA
:1018F000C8010E947B048DB79EB70A970FB6F89473
:101900009EBF0FBE8DBFEDB7FEB73196ADB7BEB768
:1019100012961C930E93119782EB91E0938382832E
:101920008091400590914105A0914205B0914305F9
:1019300084839583A683B78380EB90E0918780872B
:101940000E94482B8DB79EB70A960FB6F8949EBF9B
:101950000FBE8DBFC8010E945F041F910F910895B3
:101960000F931F93282F462F0BE015E0C801622F1D
:101970000E94A303C8010E947B048DB79EB74097C5
:101980000FB6F8949EBF0FBE8DBFEDB7FEB7319670
:10199000ADB7BEB712961C930E9311978AEB91E0E8
:1019A0009383828383E890E09583848380915205BA
:1019B00090915305A0915405B09155058683978366
:1019C000A087B18784E890E093878287809156054D
:1019D00090915705A0915805B09159058487958736
:1019E000A687B7870E94482B8DB79EB740960FB643
:1019F000F8949EBF0FBE8DBFC8010E945F041F9167
:101A00000F9108950F931F93282F462F0BE015E099
:101A1000C801622F0E94A303C8010E947B048DB7F6
:101A20009EB708970FB6F8949EBF0FBE8DBFEDB757
:101A3000FEB73196ADB7BEB712961C930E931197B1
:101A40008CEC91E0938382838FE090E09583848394
:101A500080915A05868317820E94482B8DB79EB7C6
:101A600008960FB6F8949EBF0FBE8DBFC8010E94A6
:101A70005F041F910F9108950F931F93282F462FF6
:101A80008BE095E0622F0E94A3038BE095E00E941B
:101A90007B0480915B05823018F422ED31E005C0B3
:101AA0008250823010F425ED31E000D000D000D01B
:101AB000EDB7FEB731960BE015E0ADB7BEB71296A5
:101AC0001C930E93119788ED91E093838283358365
:101AD00024830E94482B8DB79EB706960FB6F894C4
:101AE0009EBF0FBE8DBFC8010E945F041F910F9162
:101AF00008950F931F93282F462F0BE015E0C80180
:101B0000622F0E94A303C8010E947B048DB79EB779
:101B10000C970FB6F8949EBF0FBE8DBFEDB7FEB702
:101B20003196ADB7BEB712961C930E9311978BEDFD
:101B300091E09383828382EE90E095838483809109
:101B40005C0590915D05A0915E05B0915F0586836F
:101B50009783A087B1878EE890E0938782870E9461
:101B6000482B8DB79EB70C960FB6F8949EBF0FBE4C
:101B70008DBFC8010E945F041F910F9108950F93BC
:101B80001F93282F462F0BE015E0C801622F0E94FB
:101B9000A303C8010E947B048DB79EB70A970FB6B6
:101BA000F8949EBF0FBE8DBFEDB7FEB73196ADB7AF
:101BB000BEB712961C930E93119785EE91E0938316
:101BC000828380913305992787FD9095958384833F
:101BD00080EB90E09783868382EB90E0918780870B
:101BE0000E94482B8DB79EB70A960FB6F8949EBFF9
:101BF0000FBE8DBFC8010E945F041F910F91089511
:101C00000F931F93282F462F0BE015E0C801622F7A
:101C10000E94A303C8010E947B048DB79EB70A9758
:101C20000FB6F8949EBF0FBE8DBFEDB7FEB73196CD
:101C3000ADB7BEB712961C930E93119785EE91E047
:101C40009383828380913205992787FD90959583B0
:101C5000848380EB90E09783868381EB90E091878B
:101C600080870E94482B8DB79EB70A960FB6F894CE
:101C70009EBF0FBE8DBFC8010E945F041F910F91D0
:101C80000895EF92FF920F931F93282F462F8BE01A
:101C9000E82E85E0F82EC701622F0E94A303C7013A
:101CA0000E947B048DB79EB70C970FB6F8949EBF29
:101CB0000FBE8DBF0DB71EB70F5F1F4FEDB7FEB73D
:101CC000F282E1828DEE91E0F801938382838FE1CD
:101CD00090E09583848360916005709161058091A7
:101CE0006205909163050E94F73620912C05309192
:101CF0002D0540912E0550912F050E942A38F8019C
:101D000066837783808791878091310582871386E8
:101D10000E94482B8DB79EB70C960FB6F8949EBFC5
:101D20000FBE8DBFC7010E945F041F910F91FF90EE
:101D3000EF9008950F931F93282F462F0BE015E087
:101D4000C801622F0E94A303C8010E947B048DB7C3
:101D50009EB70A970FB6F8949EBF0FBE8DBFEDB722
:101D6000FEB73196ADB7BEB712961C930E9311977E
:101D700087EF91E09383828389EB90E0958384835E
:101D800080916405992787FD90959783868385E2E6
:101D900090E0918780870E94482B8DB79EB70A9666
:101DA0000FB6F8949EBF0FBE8DBFC8010E945F049E
:101DB0001F910F9108950F931F93282F462F0BE02B
:101DC00015E0C801622F0E94A303C8010E947B0492
:101DD0008DB79EB70A970FB6F8949EBF0FBE8DBF02
:101DE000EDB7FEB73196ADB7BEB712961C930E9302
:101DF000119787EF91E09383828387E890E0958342
:101E0000848380916505909166059783868385E23A
:101E100090E0918780870E94482B8DB79EB70A96E5
:101E20000FB6F8949EBF0FBE8DBFC8010E945F041D
:101E30001F910F910895EF92FF920F931F93282FF8
:101E4000462F9BE0E92E95E0F92EC701622F0E94F4
:101E5000A303C7010E947B048DB79EB70C970FB6F2
:101E6000F8949EBF0FBE8DBF0DB71EB70F5F1F4FFB
:101E7000EDB7FEB7F282E18281E092E0F801938350
:101E8000828388EE90E0958384836091EC02709168
:101E9000ED028091EE029091EF02209128053091A1
:101EA000290540912A0550912B050E942A38F801F6
:101EB0006683778380879187809130058287138638
:101EC0000E94482B8DB79EB70C960FB6F8949EBF14
:101ED0000FBE8DBFC7010E945F041F910F91FF903D
:101EE000EF900895EF92FF920F931F93282F462FA4
:101EF0003BE0E32E35E0F32EC701622F0E94A303DF
:101F0000C7010E947B048DB79EB70C970FB6F8945B
:101F10009EBF0FBE8DBF0DB71EB70F5F1F4FEDB732
:101F2000FEB7F282E18281E092E0F801938382833E
:101F300089EE90E09583848360917A0570917B05AA
:101F400080917C0590917D0520912805309129058F
:101F500040912A0550912B050E942A38F80166838A
:101F600077838087918780913005828713860E94CE
:101F7000482B8DB79EB70C960FB6F8949EBF0FBE38
:101F80008DBFC7010E945F041F910F91FF90EF90DA
:101F90000895EF92FF920F931F93282F462F5BE037
:101FA000E52E55E0F52EC701622F0E94A303C7015D
:101FB0000E947B048DB79EB70C970FB6F8949EBF16
:101FC0000FBE8DBF0DB71EB70F5F1F4FEDB7FEB72A
:101FD000F282E1828DEE91E0F8019383828387EEB5
:101FE00090E09583848360917E0570917F05809158
:101FF0008005909181052091820530918305409163
:102000008405509185050E948E3520912C053091D4
:102010002D0540912E0550912F050E942A38F80178
:1020200066837783808791878091310582871386C5
:102030000E94482B8DB79EB70C960FB6F8949EBFA2
:102040000FBE8DBFC7010E945F041F910F91FF90CB
:10205000EF9008950F931F93282F462F0BE015E064
:10206000C801622F0E94A303C8010E947B048DB7A0
:102070009EB70C970FB6F8949EBF0FBE8DBFEDB7FD
:10208000FEB73196ADB7BEB712961C930E9311975B
:1020900081E092E09383828386E190E0958384835C
:1020A0008091860590918705A0918805B09189055A
:1020B00086839783A087B18788E890E0938782879B
:1020C0000E94482B8DB79EB70C960FB6F8949EBF12
:1020D0000FBE8DBFC8010E945F041F910F9108952C
:1020E000EF92FF920F931F93282F462F6BE0E62E5F
:1020F00065E0F62EC701622F0E94A303C7010E946C
:102100007B048DB79EB70C970FB6F8949EBF0FBE99
:102110008DBF0DB71EB70F5F1F4FEDB7FEB7F28231
:10212000E1828DEE91E0F8019383828386EE90E068
:102130009583848360917E0570917F0580918005F1
:102140009091810520912C0530912D0540912E050F
:1021500050912F050E942A38F80166837783808783
:10216000918780913105828713860E94482B8DB715
:102170009EB70C960FB6F8949EBF0FBE8DBFC701D9
:102180000E945F041F910F91FF90EF900895EF92CE
:10219000FF920F931F93282F462F7BE0E72E75E0C9
:1021A000F72EC701622F0E94A303C7010E947B0480
:1021B0008DB79EB70C970FB6F8949EBF0FBE8DBF1C
:1021C0000DB71EB70F5F1F4FEDB7FEB7F282E1826A
:1021D0008BED91E0F8019383828384EE90E0958308
:1021E000848360918A0570918B05882777FD80959F
:1021F000982F0E94F7362AE037ED43E25CE30E9415
:102200002A38F80166837783808791878FE890E08A
:10221000938782870E94482B8DB79EB70C960FB686
:10222000F8949EBF0FBE8DBFC7010E945F041F912F
:102230000F91FF90EF900895AF92BF92CF92DF92EF
:10224000EF92FF920F931F93282F462F1BE0A12E92
:1022500015E0B12EC501622F0E94A303C5010E94A3
:102260007B048DB79EB7865490400FB6F8949EBFFE
:102270000FBE8DBF0DB71EB70F5F1F4FEDB7FEB777
:10228000B282A1828BE092E0F801938382832EE4F4
:1022900030E03583248382E590E0978386838091C4
:1022A0008C0590918D05A0918E05B0918F0580874A
:1022B0009187A287B38740EB50E0558744873787E3
:1022C000268780E590E0918B808B8091900590919E
:1022D0009105A0919205B0919305828B938BA48B6D
:1022E000B58B578B468B318F208F88E490E0938F8E
:1022F000828F8091940590919505958F848F578F4B
:10230000468F84E590E091A380A382E490E093A3BC
:1023100082A380913E0590913F0595A384A357A386
:1023200046A3B1E4CB2ED12CD1A6C0A6A5E4EA2EBB
:10233000F12CF3A6E2A66091960570919705809125
:1023400098059091990520912C0530912D0540918B
:102350002E0550912F050E942A38F80164A775A711
:1023600086A797A78091310580AB11AA88E590E0F8
:1023700093AB82ABF5AAE4AA80919A0590919B0554
:10238000A0919C05B0919D0586AB97ABA0AFB1AF76
:102390008DE690E093AF82AFD5AEC4AEF7AEE6AEB9
:1023A00060919E0570919F058091A0059091A10577
:1023B00020E030E048EC52E40E945C362091280591
:1023C0003091290540912A0550912B050E942A3809
:1023D000005C1F4FF80161937193819391938091F9
:1023E0003005808311820E94482B8DB79EB78A5B8F
:1023F0009F4F0FB6F8949EBF0FBE8DBFC5010E94C0
:102400005F041F910F91FF90EF90DF90CF90BF90EE
:10241000AF900895282F462F8BE095E0622F0E9401
:10242000A3038BE095E00E947B046091AD05709161
:10243000AE058091AF059091B00520914005309197
:10244000410540914205509143050E948E3520E0A0
:1024500030E044EB53E40E945C3620E030E040E89A
:1024600051E40E942A380E948D3820E030E040E894
:102470005FE30E948F350E94C436862F6093B105BA
:1024800067FF03C0805F8093B1058091B10561E073
:102490000E946E088BE095E00E945F0408950F9300
:1024A0001F93282F462F0BE015E0C801622F0E94D2
:1024B000A303C8010E947B0400D000D000D0EDB778
:1024C000FEB73196ADB7BEB712961C930E93119717
:1024D00088ED91E0938382838AEB95E095838483F2
:1024E0000E94482B8DB79EB706960FB6F8949EBFF4
:1024F0000FBE8DBFC8010E945F041F910F91089508
:10250000CF92DF92EF92FF920F931F93282F462FC7
:102510008BE095E0622F0E94A3038BE095E00E9480
:102520007B048091C305282F30E03093F102209383
:10253000F00280917705882359F50091C40510E0D9
:10254000201B310BB901882777FD8095982F0E94B9
:10255000F7366B017C016091C50570E0601B710B63
:10256000882777FD8095982F0E94F7369B01AC0154
:10257000C701B6010E945C3620E030E048EC52E42E
:102580000E942A380E94C4367093F1026093F002D0
:102590008091F0029091F1028D599F4F34F48DE9B2
:1025A0009FEF9093F1028093F0028DB79EB70A9748
:1025B0000FB6F8949EBF0FBE8DBFEDB7FEB7319634
:1025C0000BE015E0ADB7BEB712961C930E931197B2
:1025D0008FE592E09383828381EE90E095838483FC
:1025E0008091F0029091F1029783868385E290E0DA
:1025F000918780870E94482B8DB79EB70A960FB6A9
:10260000F8949EBF0FBE8DBFC8010E945F041F914A
:102610000F91FF90EF90DF90CF900895CF93DF93CD
:10262000282F462FCBE0D5E0CE01622F0E94A303D6
:10263000CE010E947B0480914505813079F400D061
:1026400000D0EDB7FEB7D283C1838BEF90E09483C7
:1026500083830E94372B109245050CC000D000D018
:10266000EDB7FEB7D283C18388EF90E09483838374
:102670000E94372B0F900F900F900F908BE095E0FA
:102680000E945F04DF91CF9108950F931F93282F2D
:10269000462F0BE015E0C801622F0E94A303C8017A
:1026A0000E947B0400D000D0EDB7FEB712830183F7
:1026B0008EEF90E0948383830E94372B0F900F90CE
:1026C0000F900F90C8010E945F041F910F91089511
:1026D000CF92DF92EF92FF920F931F937C01D62E41
:1026E000C72E0BE015E0C8016E2D4D2D0E94A303EF
:1026F000C8010E947B0400D000D0EDB7FEB7128362
:10270000018384E791E0948383830E94372BEDB7A4
:10271000FEB71283018384E691E0948383830E9451
:10272000372BEDB7FEB71283018384E591E09483E4
:1027300083830E94372BEDB7FEB71283018384E4B5
:1027400091E0948383830E94372BEDB7FEB7128309
:10275000018385E391E0948383830E94372B0F905C
:102760000F900F900F90C8010E945F04C70101965F
:102770006D2D7C2D0E9434091F910F91FF90EF90D9
:10278000DF90CF9008950F931F93282F462F0BE0D3
:1027900015E0C801622F0E94A303C8010E947B04B8
:1027A00000D000D0EDB7FEB71283018384E891E03A
:1027B000948383830E94372B0F900F900F900F907C
:1027C000C8010E945F041F910F9108950F931F93FA
:1027D0000BE015E0C80167E044E00E94A303C801D4
:1027E0000E947B0400D000D0EDB7FEB712830183B6
:1027F0008AEC91E0948383830E94372B0F900F9093
:102800000F900F90C8010E945F041F910F910895CF
:10281000EF92FF920F931F93F82EE62E0E94E6137D
:102820000BE015E0C8016F2D4E2D0E94A303C801D7
:102830000E947B0400D000D0EDB7FEB71283018365
:1028400083E191E0948383830E94372B0F900F9054
:102850000F900F90C8010E945F041F910F91FF908D
:10286000EF900895EF92FF920F931F93282F462F1A
:102870000BE0E02E05E0F02EC701622F0E94A303BB
:10288000C7010E947B040E94163428EE33E040E02A
:1028900050E00E946339CA01B9010E94F536609385
:1028A000E8027093E9028093EA029093EB020E949F
:1028B000C4368B019C018DB79EB70C970FB6F89468
:1028C0009EBF0FBE8DBFEDB7FEB73196ADB7BEB799
:1028D0001296FC92EE92119787E692E093838283A0
:1028E00083EB90E095838483C8016CE370E00E94E1
:1028F0005039CB016CE370E00E9450399783868396
:102900008AE390E091878087C8016CE370E00E94C1
:102910005039938782870E94482B8DB79EB70C96BB
:102920000FB6F8949EBF0FBE8DBFC7010E945F0413
:102930001F910F91FF90EF9008952F923F924F9229
:102940005F926F927F928F929F92AF92BF92CF923F
:10295000DF92EF92FF920F931F93DF93CF93CDB748
:10296000DEB76B970FB6F894DEBF0FBECDBF282F32
:10297000462F8BE095E0622F0E94A3038BE095E049
:102980000E947B040E9416342091670530916805EF
:102990004091690550916A0526173707480759077E
:1029A00008F09BC180916B05882391F080936C05A2
:1029B00010926B0581E080936D050E941634609340
:1029C0006E0570936F05809370059093710521C11A
:1029D0000E941634605177428040904020916E05ED
:1029E00030916F054091700550917105261737079A
:1029F0004807590710F410926D0580916C05E82E78
:102A0000FF24FA82E982F0905B05FD8690906B05C9
:102A1000A090EC02B090ED02C090EE02D090EF02D8
:102A2000409028055090290560902A0570902B054C
:102A30002091720530E04091730560915C057091C2
:102A40005D0580915E0590915F0569877A878B8728
:102A50009C879091740580916405A82FBB27A7FDE2
:102A6000B095B887AF8380917505E82FF0E0FE83BD
:102A7000ED832090F0023090F10280917605E82EEF
:102A8000FF24FC82EB828090770509811A811B8FDD
:102A90000A8FE42EFF2400E010E0EE86FF86088B0C
:102AA000198B492F50E060E070E04A8B5B8B6C8B98
:102AB0007D8BB901882777FD8095982F6E8B7F8B52
:102AC000888F998FA1C08A8D9B8D01969B8F8A8F4D
:102AD00006972CF0A1E0B0E0BB8FAA8F1BC0EA8D57
:102AE000FB8DE330F10509F441C0E430F1053CF41D
:102AF000E130F10579F0329709F07FC012C00A8DFC
:102B00001B8D0430110509F44AC00530110509F088
:102B100074C065C01D85123008F06FC0992493946D
:102B20006CC0C601B501A30192010E942A387B0145
:102B30008C016E897F89888D998D0E94F7369B0163
:102B4000AC01C801B7010E94553688230CF055C06E
:102B5000C601B50129E23CE54FE85FE30E941F385A
:102B600018160CF04AC052E0952E47C0C601B501B8
:102B7000A30192010E942A387B018C016E857F851A
:102B8000888999890E94F5369B01AC01C801B7017B
:102B90000E941F3818168CF543E0942E2EC06A89C7
:102BA0007B898C899D890E94F53620E030E040E2E7
:102BB00051E40E945C369B01AC0169857A858B8566
:102BC0009C850E94553687FD07C02F8138854D8131
:102BD0005E81241735078CF434E0932E0EC06B8190
:102BE0007C81261637064CF47DE927167FEF3706E1
:102BF00021F0882011F425E0922E8A8D9B8DA981E9
:102C0000BA818A179B0719F0992009F45CCF90923A
:102C10006B050E94163468517C4F8F4F9F4F609315
:102C20006705709368058093690590936A058091A4
:102C30006D05813051F480917805813021F48BE06D
:102C400095E00E94C8041092780580917905882348
:102C500019F42DE732E023C080916B058230A1F09A
:102C6000833028F4882351F08130C9F40AC08430BD
:102C700089F0843060F0853091F40FC02AE832E0AA
:102C80000EC027E932E00BC024EA32E008C021EB95
:102C900032E005C02EEB32E002C02BEC32E000D077
:102CA00000D000D0EDB7FEB731968BE095E0ADB720
:102CB000BEB712969C938E93119788ED91E0938303
:102CC0008283358324830E94482BEDB7FEB7369666
:102CD0000FB6F894FEBF0FBEEDBF8BE095E00E94EB
:102CE0005F046B960FB6F894DEBF0FBECDBFCF91D9
:102CF000DF911F910F91FF90EF90DF90CF90BF90E9
:102D0000AF909F908F907F906F905F904F903F908B
:102D10002F900895EF92FF920F931F938091A20539
:102D2000843009F068C080913805813041F4809189
:102D300039058B3009F438C1813051F435C1823006
:102D400009F032C1809139058650823008F42CC1D7
:102D5000909139058091A3058917A1F19093A3055E
:102D60000E9416346093A4057093A5058093A60570
:102D70009093A7059091A3058091F202981711F501
:102D800080917805813091F0813018F08230B1F473
:102D900013C011E0109378050E94163461567A4EE4
:102DA0008040904030F41093A80508C082E08093E2
:102DB00078051092A80502C0109278058BE095E086
:102DC0000E94C8040E9416342091A4053091A505E4
:102DD0004091A6055091A705621B730B840B950BC0
:102DE000615D77408040904008F4DEC080913905F5
:102DF0008093F202D9C0853029F48091F30290913A
:102E0000F40214C0863029F48091F5029091F60204
:102E10000DC0873029F48091F7029091F80206C026
:102E2000883041F48091F9029091FA029093AA05BA
:102E30008093A9058091AB052091A9053091AA0541
:102E4000882309F04DC0B7E029303B07C8F00E9445
:102E5000163461567A4E8040904020F481E0809391
:102E6000A8050CC08091A805813041F080916D05C6
:102E7000813021F08BE095E00E94C80482E02DC0F3
:102E800084E0203B380768F480917805882349F076
:102E90001092A8058BE095E00E94C8041092780576
:102EA00083C0205B34402955324008F07DC08091BA
:102EB000AC05863009F478C080917805813009F43A
:102EC00073C080916D05813009F46EC01092A80521
:102ED0008BE095E00E94C80481E08093780564C08F
:102EE000215B344008F460C00E94163461567A4E6B
:102EF0008040904008F041C08091A8058130E9F100
:102F0000E090A405F090A5050091A6051091A705F5
:102F100088EE93E0A0E0B0E0E80EF91E0A1F1B1F48
:102F20000E941634E616F70608071907E8F581E04F
:102F30008093A80517C01092A8058BE095E00E9429
:102F4000C80480917805823019F41092780503C086
:102F50008F5F8093780580917805823018F082E049
:102F6000809378050E9416346093A4057093A5059C
:102F70008093A6059093A70517C0E090A405F09054
:102F8000A5050091A6051091A70588EE93E0A0E0A5
:102F9000B0E0E80EF91E0A1F1B1F0E941634E61649
:102FA000F7060807190738F21F910F91FF90EF906D
:102FB00008958BE095E00E94C8040E94E6130E94E9
:102FC0005C070895CF93DF93AC01E091B205F091D7
:102FD000B3052091B4053091B505C9018C599F4FB7
:102FE0008E179F0714F0EA0102C0EA0121972456C8
:102FF0003040E217F3070CF42196842F90E0C817B5
:10300000D90749F08091AC05882329F086E796E03E
:103010004C2F0E940032CE01DF91CF910895EF92A4
:10302000FF920F931F930E941634209167053091F1
:1030300068054091690550916A05261737074807CA
:10304000590708F03BC10E9416346C507E4F8F4FD9
:103050009F4F60936705709368058093690590930F
:103060006A058BE095E00E94C8048BE095E065E07E
:1030700047E00E94A3038BE095E00E947B048091CF
:10308000B4059091B505892BB1F48091B605909166
:10309000B705892B81F48091B2059091B305909387
:1030A000B5058093B4058091B8059091B9059093CA
:1030B000B7058093B6052091B8053091B9054091C8
:1030C000B6055091B705C901845690404817590775
:1030D00024F48091AC058F5F08C02C593F4F241712
:1030E00035072CF48091AC0581508093AC0580911C
:1030F000AC0587FF03C01092AC0505C083301CF0FF
:1031000082E08093AC058091AC05813009F443C026
:10311000823009F47DC0882309F0D0C000D000D0EF
:103120000BE015E0ADB7BEB712961C930E93119746
:1031300081EB91E014969C938E9313970E94372B0A
:1031400000D000D0EDB7FEB73196ADB7BEB712963E
:103150001C930E93119788ED92E093838283809164
:1031600073058483158280913005868317820E94BF
:10317000482BEDB7FEB738960FB6F894FEBF0FBEDA
:10318000EDBF8091730590E06CE773E00E94E21759
:103190008093730593C000D000D00BE015E0ADB76D
:1031A000BEB712961C930E9311978FE991E0149677
:1031B0009C938E9313970E94372B00D000D0EDB7CD
:1031C000FEB73196ADB7BEB712961C930E9311970A
:1031D00088ED92E0938382838091720584831582C7
:1031E00080913005868317820E94482BEDB7FEB789
:1031F00038960FB6F894FEBF0FBEEDBF80917205F2
:1032000090E06EE773E00E94E2178093720556C06B
:1032100000D000D06BE0E62E65E0F62EADB7BEB76D
:103220001296FC92EE9211978EE891E014969C9380
:103230008E9313970E94372BEDB7FEB738970FB6D2
:10324000F894FEBF0FBEEDBF0DB71EB70F5F1F4F47
:10325000F282E18280EE92E0D80113969C938E93E5
:1032600012976091740570E080E090E00E94F5365E
:1032700020E030E040E251E40E945C36F8016483D3
:1032800075838683978386E790E09187808780E2C5
:1032900090E0938782870E94482B8DB79EB70C964B
:1032A0000FB6F8949EBF0FBE8DBF8091740590E05D
:1032B00060E873E00E94E217809374058BE095E06C
:1032C0000E945F041F910F91FF90EF900895EF927D
:1032D000FF920F931F930E9416340E94F5367B01D4
:1032E0008C016091C6057091C7058091C8059091C9
:1032F000C90520E030E849E055E40E948F359B0184
:10330000AC01C801B7010E94553688230CF0A7C252
:103310008091A205843010F00E948A168091A80541
:10332000882309F099C280917805823009F475C22A
:10333000A82FB0E0FD01E059FB4F808180FF0BC05A
:10334000FD01EC52FB4F6081AE52BB4F8C9190E07F
:1033500070E00E949D1480917805A82FB0E0FD01D7
:10336000E659FB4F808180FF0BC0FD01EC58FB4FFD
:103370006081AE58BB4F8C9190E070E00E94C31307
:1033800080917805A82FB0E0FD01E659FB4F8081C0
:1033900081FF0BC0FD01E858FB4F6081AA58BB4F6D
:1033A0008C9190E070E00E94000E80917805A82F2B
:1033B000B0E0FD01E659FB4F808182FF0BC0FD01AB
:1033C000E458FB4F6081A658BB4F8C9190E070E0B1
:1033D0000E94BF0D80917805A82FB0E0FD01E6594D
:1033E000FB4F808183FF0BC0FD01E058FB4F6081E4
:1033F000A258BB4F8C9190E070E00E94790D8091B3
:103400007805A82FB0E0FD01E659FB4F808185FFCC
:103410000BC0FD01EC57FB4F6081AE57BB4F8C9149
:1034200090E070E00E94020D80917805A82FB0E036
:10343000FD01E659FB4F808186FF0BC0FD01E85777
:10344000FB4F6081AA57BB4F8C9190E070E00E94C7
:103450003C0D80917805A82FB0E0FD01E659FB4FA7
:10346000808187FF0BC0FD01E457FB4F6081A657A9
:10347000BB4F8C9190E070E00E94B00C8091780579
:10348000A82FB0E0FD01E659FB4F808184FF0BC0FF
:10349000FD01E057FB4F6081A257BB4F8C9190E03C
:1034A00070E00E949A0E80917805A82FB0E0FD018F
:1034B000E459FB4F808180FF0BC0FD01EC56FB4FB0
:1034C0006081AE56BB4F8C9190E070E00E942C0C56
:1034D00080917805A82FB0E0FD01E459FB4F808171
:1034E00081FF0BC0FD01E856FB4F6081AA56BB4F20
:1034F0008C9190E070E00E946E0C80917805A82F6E
:10350000B0E0FD01E459FB4F808182FF0BC0FD015B
:10351000E456FB4F6081A656BB4F8C9190E070E063
:103520000E940E138091CA05813051F58091780573
:10353000A82FB0E0FD01E459FB4F808184FF0BC050
:10354000FD01EC55FB4F6081AE55BB4F8C9190E077
:1035500070E00E94410E80917805A82FB0E0FD0137
:10356000E459FB4F808183FF0BC0FD01E056FB4F08
:103570006081A256BB4F8C9190E070E00E94700B6E
:1035800080917805A82FB0E0FD01E459FB4F8081C0
:1035900087FF0BC0FD01E055FB4F6081A255BB4F7B
:1035A0008C9190E070E00E94321480917805A82FF1
:1035B000B0E0FD01E459FB4F808185FF0BC0FD01A8
:1035C000E855FB4F6081AA55BB4F8C9190E070E0AD
:1035D0000E94E50B80917805A82FB0E0FD01E45929
:1035E000FB4F808186FF0BC0FD01E455FB4F6081DE
:1035F000A655BB4F8C9190E070E00E94880B8091A3
:103600007805A82FB0E0FD01E259FB4F808182FFD1
:103610000BC0FD01E854FB4F6081AA54BB4F8C9155
:1036200090E070E00E94701080917805A82FB0E0C3
:10363000FD01E259FB4F808187FF0BC0FD01E4547F
:10364000FB4F6081A654BB4F8C9190E070E00E94CC
:10365000C90F80917805A82FB0E0FD01E259FB4F1A
:10366000808183FF0BC0FD01E054FB4F6081A254B9
:10367000BB4F8C9190E070E00E94720F80917805B2
:10368000A82FB0E0FD01E259FB4F808181FF0BC004
:10369000FD01EC53FB4F6081AE53BB4F8C9190E02A
:1036A00070E00E941B0F80917805A82FB0E0FD010B
:1036B000E259FB4F808184FF0BC0FD01E853FB4FB3
:1036C0006081AA53BB4F8C9190E070E00E94DB0EAA
:1036D00080917805A82FB0E0FD01E259FB4F808171
:1036E00085FF0BC0FD01E453FB4F6081A653BB4F28
:1036F0008C9190E070E00E94A40A80917805A82F38
:10370000B0E0FD01E259FB4F808186FF0BC0FD0157
:10371000E053FB4F6081A253BB4F8C9190E070E06F
:103720000E94681380917805A82FB0E0FD01E2594E
:10373000FB4F808180FF0BC0FD01EC54FB4F60818B
:10374000AE54BB4F8C9190E070E00E94C710809106
:103750007805A82FB0E0FD01E059FB4F808182FF82
:103760000BC0FD01E852FB4F6081AA52BB4F8C9108
:1037700090E070E00E940A1280917805A82FB0E0D6
:10378000FD01E059FB4F808183FF0BC0FD01E45236
:10379000FB4F6081A652BB4F8C9190E070E00E947D
:1037A0002A1080917805A82FB0E0FD01E059FB4F69
:1037B000808184FF0BC0FD01E052FB4F6081A2526B
:1037C000BB4F8C9190E070E00E941C1180917805B5
:1037D000A82FB0E0FD01E059FB4F808186FF0BC0B0
:1037E000FD01E851FB4F6081AA51BB4F8C9190E0E5
:1037F00070E00E94801280917805A82FB0E0FD0152
:10380000E059FB4F808185FF37C0FD01E451FB4F3C
:103810006081A651BB4F8C911AC08091700480FFCB
:1038200008C06091D4048091D20490E070E00E94BE
:103830009D148091700485FF1FC0E0917805F0E031
:10384000DF01A451BB4F6C91E651FB4F808190E0AA
:1038500070E00E944F1210C00E940F180DC08BE044
:1038600095E00E94C80481E08093FB0285E090E02F
:103870006AE070E00E9408141F910F91FF90EF9092
:103880000895CF93DF93EC018BE095E00E949F03B6
:10389000C817D9073CF08BE095E00E949403892B70
:1038A00009F42397CE01DF91CF910895EF92FF9213
:1038B0000F931F93CF93DF930091780510E08AEF69
:1038C00090E0089F7001099FF00C189FF00C1124E4
:1038D000C7010E941008F801E659FB4F882319F030
:1038E0008081816002C080818E7F80838091780595
:1038F000C82FD0E0C70102960E941008CE58DB4FB7
:10390000888380917805C82FD0E0C70104960E9473
:10391000100890E00E94411CCC58DB4F8883009136
:10392000780510E0C70188569F4F0E941008F801E3
:10393000E659FB4F882319F08081806102C08081A5
:103940008F7E808380917805C82FD0E0C70186568E
:103950009F4F0E941008C257DB4F888380917805E3
:10396000C82FD0E0C70184569F4F0E94100890E0F6
:103970000E94411CC057DB4F88830091780510E0FE
:10398000C70106960E941008F801E659FB4F8823EC
:1039900019F08081826002C080818D7F8083809158
:1039A0007805C82FD0E0C70108960E941008CA58B1
:1039B000DB4F888380917805C82FD0E0C7010A9635
:1039C0000E94100890E00E94411CC858DB4F888379
:1039D0000091780510E0C7010C960E941008F801CC
:1039E000E659FB4F882319F08081846002C08081F2
:1039F0008B7F808380917805C82FD0E0C7010E9619
:103A00000E941008C658DB4F888380917805C82F24
:103A1000D0E0C70140960E94100890E00E94411C2F
:103A2000C458DB4F88830091780510E0C7014296A7
:103A30000E941008F801E659FB4F882319F0808195
:103A4000886002C08081877F808380917805C82F3D
:103A5000D0E0C70144960E941008C258DB4F88830B
:103A600080917805C82FD0E0C70146960E941008C3
:103A700090E00E94411CC058DB4F8883009178057C
:103A800010E0C7014E960E941008F801E659FB4F5E
:103A9000882319F08081806202C080818F7D8083BD
:103AA00080917805C82FD0E0C70180960E94100849
:103AB000CE57DB4F888380917805C82FD0E0C701AF
:103AC00082960E94100890E00E94411CCC57DB4F68
:103AD00088830091780510E0C70184960E94100841
:103AE000F801E659FB4F882319F08081806402C0F9
:103AF00080818F7B808380917805C82FD0E0C701BB
:103B000086960E941008CA57DB4F888380917805FB
:103B1000C82FD0E0C70188960E94100890E00E944C
:103B2000411CC857DB4F88830091780510E0C7011E
:103B30008A960E941008F801E659FB4F882319F075
:103B40008081806802C080818F7780838091780532
:103B5000C82FD0E0C7018C960E941008C657DB4FD3
:103B6000888380917805C82FD0E0C7018E960E9487
:103B7000100890E00E94411CC457DB4F88830091DD
:103B8000780510E0C701C0960E941008F801E459BA
:103B9000FB4F882319F08081816002C080818E7F75
:103BA000808380917805C82FD0E0C701C2960E941B
:103BB0001008CE56DB4F888380917805C82FD0E05F
:103BC000C701C4960E94100890E00E94411CCC5688
:103BD000DB4F88830091780510E0C701C6960E94EC
:103BE0001008F801E459FB4F882319F080818260A6
:103BF00002C080818D7F808380917805C82FD0E0BE
:103C0000C701C8960E941008CA56DB4F888380916E
:103C10007805C82FD0E0C701CA960E94100890E02E
:103C20000E94411CC856DB4F88830091780510E044
:103C3000C701CC960E941008F801E459FB4F882375
:103C400019F08081846002C080818B7F80838091A5
:103C50007805C82FD0E0C701CE960E941008C6563E
:103C6000DB4F888380917805C82FD0E0C701805C46
:103C70009F4F0E94100890E00E94411CC456DB4FE9
:103C800088830091780510E0C701885B9F4F0E94F0
:103C90001008F801E459FB4F882319F080818061F6
:103CA00002C080818F7E808380917805C82FD0E00C
:103CB000C701865B9F4F0E941008CE55DB4F88835B
:103CC00080917805C82FD0E0C701845B9F4F0E9488
:103CD000100890E00E94411CCC55DB4F8883009176
:103CE000780510E0C7018E5B9F4F0E941008F80115
:103CF000E459FB4F882319F08081886002C08081DD
:103D0000877F808380917805C82FD0E0C7018C5BC6
:103D10009F4F0E941008C256DB4F88838091780520
:103D2000C82FD0E0C7018A5B9F4F0E94100890E027
:103D30000E94411CC056DB4F88830091780510E03B
:103D4000C701805B9F4F0E941008F801E459FB4FA8
:103D5000882319F08081806202C080818F7D8083FA
:103D600080917805C82FD0E0C7018E5A9F4F0E94DE
:103D70001008CA55DB4F888380917805C82FD0E0A2
:103D8000C7018C5A9F4F0E94100890E00E94411C6E
:103D9000C855DB4F88830091780510E0C7018A5A27
:103DA0009F4F0E941008F801E459FB4F882319F037
:103DB0008081806402C080818F7B808380917805C0
:103DC000C82FD0E0C701885A9F4F0E941008C655DF
:103DD000DB4F888380917805C82FD0E0C701865AD1
:103DE0009F4F0E94100890E00E94411CC455DB4F79
:103DF00088830091780510E0C70182569F4F0E948A
:103E00001008F801E459FB4F882319F0808180687D
:103E100002C080818F77808380917805C82FD0E0A1
:103E2000C70180569F4F0E941008C255DB4F888300
:103E300080917805C82FD0E0C7018E559F4F0E9412
:103E4000100890E00E94411CC055DB4F8883009110
:103E5000780510E0C7018E599F4F0E941008F801A5
:103E6000E259FB4F882319F08081816002C0808174
:103E70008E7F808380917805C82FD0E0C7018C5950
:103E80009F4F0E941008CE54DB4F888380917805A5
:103E9000C82FD0E0C7018A599F4F0E94100890E0B8
:103EA0000E94411CCC54DB4F88830091780510E0C0
:103EB000C70182599F4F0E941008F801E259FB4F39
:103EC000882319F08081846002C080818B7F808389
:103ED00080917805C82FD0E0C70180599F4F0E947C
:103EE0001008CA54DB4F888380917805C82FD0E032
:103EF000C7018E589F4F0E94100890E00E94411CFD
:103F0000C854DB4F88830091780510E0C7018457BF
:103F10009F4F0E941008F801E259FB4F882319F0C7
:103F20008081806802C080818F778083809178054E
:103F3000C82FD0E0C70182579F4F0E941008C65477
:103F4000DB4F888380917805C82FD0E0C701805768
:103F50009F4F0E94100890E00E94411CC454DB4F08
:103F600088830091780510E0C7018E569F4F0E940C
:103F70001008F801E259FB4F882319F08081826014
:103F800002C080818D7F808380917805C82FD0E02A
:103F9000C7018C569F4F0E941008CE53DB4F888379
:103FA00080917805C82FD0E0C7018A569F4F0E94A4
:103FB000100890E00E94411CCC53DB4F8883009195
:103FC000780510E0C7018C589F4F0E941008F80137
:103FD000E259FB4F882319F08081886002C08081FC
:103FE000877F808380917805C82FD0E0C7018A58E9
:103FF0009F4F0E941008C254DB4F88838091780540
:10400000C82FD0E0C70188589F4F0E94100890E049
:104010000E94411CC054DB4F88830091780510E05A
:10402000C70186589F4F0E941008F801E259FB4FC4
:10403000882319F08081806102C080818F7E808317
:1040400080917805C82FD0E0C70184589F4F0E9407
:104050001008CA53DB4F888380917805C82FD0E0C1
:10406000C70182589F4F0E94100890E00E94411C97
:10407000C853DB4F88830091780510E0C701805852
:104080009F4F0E941008F801E259FB4F882319F056
:104090008081806202C080818F7D808380917805DD
:1040A000C82FD0E0C7018E579F4F0E941008C653FB
:1040B000DB4F888380917805C82FD0E0C7018C57EB
:1040C0009F4F0E94100890E00E94411CC453DB4F98
:1040D00088830091780510E0C7018A579F4F0E949E
:1040E0001008F801E259FB4F882319F080818064A1
:1040F00002C080818F7B808380917805C82FD0E0BB
:10410000C70188579F4F0E941008C253DB4F888316
:1041100080917805C82FD0E0C70186579F4F0E9435
:10412000100890E00E94411CC053DB4F888300912F
:10413000780510E0C7018C559F4F0E941008F801C8
:10414000E059FB4F882319F08081816002C0808193
:104150008E7F808380917805C82FD0E0C7018A5573
:104160009F4F0E941008CE52DB4F888380917805C4
:10417000C82FD0E0C70188559F4F0E94100890E0DB
:104180000E94411CCC52DB4F88830091780510E0DF
:10419000C70180559F4F0E941008F801E059FB4F5E
:1041A000882319F08081846002C080818B7F8083A6
:1041B00080917805C82FD0E0C7018E549F4F0E9490
:1041C0001008CA52DB4F888380917805C82FD0E051
:1041D000C7018C549F4F0E94100890E00E94411C20
:1041E000C852DB4F88830091780510E0C7018A54DC
:1041F0009F4F0E941008F801E059FB4F882319F0E7
:104200008081886002C08081877F8083809178056B
:10421000C82FD0E0C70188549F4F0E941008C65293
:10422000DB4F888380917805C82FD0E0C701865482
:104230009F4F0E94100890E00E94411CC452DB4F27
:1042400088830091780510E0C70184549F4F0E9435
:104250001008F801E059FB4F882319F08081806134
:1042600002C080818F7E808380917805C82FD0E046
:10427000C70182549F4F0E941008C252DB4F8883AF
:1042800080917805C82FD0E0C70180549F4F0E94CD
:10429000100890E00E94411CC052DB4F88830091BF
:1042A000780510E0C7018E539F4F0E941008F80157
:1042B000E059FB4F882319F08081806802C080811B
:1042C0008F77808380917805C82FD0E0C7018C5309
:1042D0009F4F0E941008CE51DB4F88838091780554
:1042E000C82FD0E0C7018A539F4F0E94100890E06A
:1042F0000E94411CCC51DB4F88830091780510E06F
:10430000C70188539F4F0E941008F801E059FB4FE6
:10431000882319F08081806202C080818F7D808334
:1043200080917805C82FD0E0C70186539F4F0E9427
:104330001008C651DB4F888380917805C82FD0E0E4
:10434000C70184539F4F0E94100890E00E94411CB7
:10435000C451DB4F8883DF91CF911F910F91FF9064
:10436000EF9008958F929F92AF92BF92CF92DF927B
:10437000FF920F931F93CF93DF93F62E4901C82E20
:10438000DD248601000F111F5801AC0CBD1CE50196
:10439000CC0FDD1FCC0FDD1FC55BD94F18828B8181
:1043A0009C818430910509F48EC0853091055CF4C0
:1043B0008230910509F443C0833091050CF0BFC0F1
:1043C0009923C4F44FC28730910509F443C1883062
:1043D000910544F48530910509F4DEC0069709F093
:1043E00041C207C18830910509F47AC1099709F0E3
:1043F00039C2E7C18EEF681709F034C282E090E05D
:104400009C838B8380E790E0C89ED001C99EB00D4D
:10441000D89EB00D1124A552BA4F13961C92139733
:1044200088E390E0C89EF001C99EF00DD89EF00D83
:104430001124EE0FFF1FE352FA4F6083A4C1E5E69B
:10444000E61788F489818F5F8983F501EE0FFF1FDE
:10445000EE0FFF1FE35BF94F80818F5F808318822F
:1044600081E090E02DC080E790E0C89EF001C99EF9
:10447000F00DD89EF00D1124E552FA4F63831D8292
:1044800080818627282F2295207F282730E0522FF1
:104490004427C90163E0880F991F6A95E1F748270F
:1044A0005927818190E04827592784E03595279541
:1044B0008A95E1F7422753275183408384E090E0B7
:1044C0009C838B83CFC18CE190E0C89EF001C99E94
:1044D000F00DD89EF00D1124EE0FFF1FEE0FFF1F01
:1044E000E152FA4F608380E790E0C89EF001C99ED8
:1044F000F00DD89EF00D1124E552FA4F80818627E9
:10450000282F2295207F282730E0522F4427C901E9
:10451000B3E0880F991FBA95E1F7482759278181A1
:1045200090E048275927A4E035952795AA95E1F70B
:10453000422753275183408383E090E0C1CF80E737
:1045400090E0C89EF001C99EF00DD89EF00D112498
:10455000E552FA4F658380818627282F2295207F98
:10456000282730E0522F4427C90163E0880F991FA4
:104570006A95E1F748275927818190E04827592714
:1045800004E0359527950A95E1F742275327518393
:10459000408385E090E094CF80E790E0C89EF001F2
:1045A000C99EF00DD89EF00D1124E552FA4F668396
:1045B00080818627282F2295207F282730E0522FC0
:1045C0004427C901B3E0880F991FBA95E1F748273E
:1045D0005927818190E048275927A4E035952795F0
:1045E000AA95E1F7422753275183408386E090E064
:1045F00067CF80E790E0C89EF001C99EF00DD89E7D
:10460000F00D1124E552FA4F678380818627282F09
:104610002295207F282730E0522F4427C90163E0EC
:10462000880F991F6A95E1F748275927818190E003
:104630004827592794E0359527959A95E1F7422721
:104640005327518340838381882309F446C087E040
:1046500090E036CF6D81F80183E0EE0FFF1F8A9561
:10466000E1F7E01BF10B319603E0EE0FFF1F0A9517
:10467000E1F7E60FF11DE552FA4FF0826F5F6D83AF
:1046800080E790E0C89EF001C99EF00DD89EF00D25
:104690001124E552FA4F80818F25282F2295207F03
:1046A000282730E0522F4427C901B3E0880F991F13
:1046B000BA95E1F748275927818190E04827592783
:1046C000A4E035952795AA95E1F742275327518312
:1046D00040838381681709F0C5C088E090E0F0CE80
:1046E00080E790E0C89ED001C99EB00DD89EB00D65
:1046F0001124A552BA4F9C911796EC911797F0E0B0
:10470000E65EFC4F80818927482F4295407F4827ED
:1047100050E0342F2227CA0173E0880F991F7A9541
:10472000E1F72827392711968C91119790E02827D7
:10473000392764E0559547956A95E1F72427352791
:1047400011963C932E938F2D90E030708217930733
:10475000F9F0F501EE0FFF1FEE0FFF1FE35BF94FBE
:1047600080818F5F8083188281E090E09C838B83BF
:10477000FEEFFF1609F076C082E090E09C838B8309
:1047800013961C9213978FEF9FEF8D939C936AC0A3
:1047900089E090E09C838B83F80183E0EE0FFF1F9C
:1047A0008A95E1F7E01BF10B319613E0EE0FFF1F46
:1047B0001A95E1F78D81E80FF11DE552FA4FF0826D
:1047C00051C0262F30E080E790E0C89EB001C99E1E
:1047D000700DD89E700D112465527A4FFB018181B6
:1047E00090E028173907E9F0F501EE0FFF1FEE0FF3
:1047F000FF1FE35BF94F80818F5F8083188281E028
:1048000090E09C838B83FEEFFF1661F582E090E0E1
:104810009C838B83EB011B828FEF9FEF99838883AF
:1048200021C081E0888381E090E09C838B83F80144
:10483000A3E0EE0FFF1FAA95E1F7E01BF10B319605
:1048400033E0EE0FFF1F3A95E1F78D81E80FF11D80
:10485000E452FA4FF082DA01FB0180E701900D92F9
:104860008150E1F7D601AA0FBB1FAC0DBD1DAA0FE9
:10487000BB1FAA0FBB1FA55BB94F8C91813069F597
:104880008CE190E0C89EF001C99EF00DD89EF00D1D
:104890001124EE0FFF1FEE0FFF1FE152FA4F808130
:1048A00016968C93169718968D919C911997892B33
:1048B00021F41B961C921E921A97F601EE0FFF1F11
:1048C000EC0DFD1DEE0FFF1FEE0FFF1FE55BF94F17
:1048D00080859185019691878087F601EE0FFF1FF5
:1048E000EC0DFD1DEE0FFF1FEE0FFF1FDF01A55B9F
:1048F000B94F16968C9116978F5FE4018E831896A8
:104900008D919C91199799878887E35BF94F8081F6
:104910008A871B8610828C91DF91CF911F910F9116
:10492000FF90DF90CF90BF90AF909F908F900895B1
:104930004F925F927F928F929F92AF92BF92CF924F
:10494000DF92EF92FF920F931F93DF93CF93CDB738
:10495000DEB7C854D0400FB6F894DEBF0FBECDBF4F
:104960000BE015E0C8010E94C804C80166E049E0F8
:104970000E94A303C8010E947B0400D000D0EDB7C1
:10498000FEB7128301838EE092E0948383830E94BA
:10499000372B0F900F900F900F90C8010E945F046B
:1049A00000D000D00EEE14E0EDB7FEB71283018305
:1049B0008EEF91E0948383830E94372B33EF432E55
:1049C00031E0532EEE24FF24CC24DD240F900F90F1
:1049D0000F900F90702E012F29E0A22EB12CAC0E5B
:1049E000BD1E4E010894811C911C8EEE94E00E9425
:1049F000EB2B982F8D3031F08D30DCF180538230ED
:104A0000C0F530C01830A1F59981892F80538230CC
:104A100078F5913311F490E801C090E08A818133F8
:104A200009F4905C8B81813309F4905E8C81813331
:104A300009F4905F8D81813309F4985F8E81813311
:104A400009F49C5F8F81813309F49E5F88858133EF
:104A500009F49F5FF501EE0DFF1D90830894E11CA2
:104A6000F11C06C0F401E10FF11D90831F5F01C02E
:104A700010E0F0E4EF16F104C9F48BE095E0B60124
:104A8000A5010E94B3030894C11CD11C00D000D022
:104A9000EDB7FEB771820283548243820E94372BA6
:104AA000EE24FF240F900F900F900F90FFEFCF1682
:104AB000D10409F00CF499CFC85BDF4F0FB6F8941E
:104AC000DEBF0FBECDBFCF91DF911F910F91FF9041
:104AD000EF90DF90CF90BF90AF909F908F907F909E
:104AE0005F904F900895AF92BF92CF92DF92EF9276
:104AF000FF920F931F93DF93CF93CDB7DEB7CC57C1
:104B0000D0400FB6F894DEBF0FBECDBF4DE0E42E0F
:104B1000F12CEC0EFD1E5E010894A11CB11CCC24EE
:104B2000C3948E010B5E1F4F01C28EEE94E00E9473
:104B3000EB2BD82E8091CB05882311F50E941634DB
:104B400060527E4480409040D8F40E9416346958E8
:104B5000734180409040A0F0FAE0DF1619F02DE09C
:104B6000D21631F48091CC058F5F8093CC0502C0C2
:104B70001092CC058091CC05833011F40E949824CA
:104B800080E06D2DA70195010E94B221882309F4D0
:104B9000C9C1C092CB058C89833209F471C18432BA
:104BA00060F4813009F449C08130B8F0883109F4EB
:104BB00064C08E3109F0B6C1DDC08E3309F408C17E
:104BC0008F3320F48A3209F0ADC155C18A3409F41B
:104BD00086C0883A09F0A6C17FC1C09245058A897E
:104BE0008093CD058B898093CE05F80184818093D5
:104BF0003805F701808580933905F8018681809317
:104C0000CF058823880F880B8C218093790510921B
:104C1000D0050E9416340E94F5366093C605709345
:104C2000C7058093C8059093C9058091FB02813028
:104C300009F078C18093D10575C1F701668977893C
:104C400080E090E00E94F53620E030E04AE754E44E
:104C50000E945C3660935C0570935D0580935E05F1
:104C600090935F05F701808D918D90938B058093D4
:104C70008A0586A18093640555C1F7016089718911
:104C8000828993890E94F73620E836E948E15BE49F
:104C90000E945C36609352057093530580935405CF
:104CA00090935505F70164897589868997890E94D3
:104CB000F73620E836E948E15BE40E945C36609311
:104CC0005605709357058093580590935905F80140
:104CD000848D80935B05858D80935A0523C1F801EF
:104CE00080819181A281B3818093EC029093ED0247
:104CF000A093EE02B093EF0284819581A681B781E3
:104D000080937A0590937B05A0937C05B0937D05F5
:104D1000F701608D718D882777FD8095982F0E940F
:104D2000F736609340057093410580934205909358
:104D30004305F701828D938D9093660580936505F9
:104D400080899189A289B38980937E0590937F059C
:104D5000A0938005B0938105F80184859585A6858B
:104D6000B7858093860590938705A0938805B093B7
:104D70008905D8C0F701608971898289938921EEFC
:104D80003EE245E652E40E942A380E94C43660930F
:104D90003205F801648175818681978121EE3EE2BA
:104DA00045E652E40E942A380E94C43660933305D7
:104DB000F801648575858685978521EE3EE245E696
:104DC00052E40E942A380E94C4366093D205AAC0D9
:104DD000F80180819181A281B38180938C059093A9
:104DE0008D05A0938E05B0938F0584819581A68152
:104DF000B7818093900590939105A0939205B0930D
:104E00009305848995899093950580939405868967
:104E1000978990933F0580933E05F70180A191A16A
:104E200090933D0580933C0580899189A289B3893F
:104E30008093960590939705A0939805B093990554
:104E4000F80184859585A685B78580939E05909306
:104E50009F05A093A005B093A105F701808D918DCA
:104E6000A28DB38D80939A0590939B05A0939C058A
:104E7000B0939D0557C0F701808580933B0552C0D4
:104E8000F801848195819093B3058093B205868162
:104E900097819093B9058093B80584859585909303
:104EA000F4028093F302868597859093F6028093AF
:104EB000F502F701808D918D9093F8028093F702AF
:104EC000F801828993899093FA028093F902F7019D
:104ED000858D8093C30526C0F80180819181A281D0
:104EE000B3818093AD059093AE05A093AF05B093C9
:104EF000B00584819581A681B78180933405909314
:104F00003505A0933605B0933705F701808991895F
:104F1000A289B3898093D3059093D405A093D50536
:104F2000B093D6058AE890E00E947D348EEE94E03E
:104F30000E94BB2B181619060CF4F7CD8091D705EB
:104F40009091D8052B853C85820F931F9093D805AF
:104F50008093D7052B818091D9059091DA05820F36
:104F6000911D9093DA058093D905C458DF4F0FB691
:104F7000F894DEBF0FBECDBFCF91DF911F910F918F
:104F8000FF90EF90DF90CF90BF90AF9008952F9259
:104F90003F924F925F926F927F928F929F92AF92C9
:104FA000BF92CF92DF92EF92FF921F93CF93DF9346
:104FB00085E090E06CE070E00E94451364EF71E0E2
:104FC00080E090E00E942434A6E42A2EA2E03A2E4B
:104FD000FEE34F2EF2E05F2EE6E36E2EE2E07E2E41
:104FE0007EE2872E72E0972E66E2A62E62E0B62E53
:104FF0005DE1C52E52E0D52EEE24FF2410E0CBE07B
:10500000D5E0C7016AEF70E00E945039892B09F0A2
:1050100091C01F5F8BE095E061E14CE00E94A3032B
:105020008BE095E00E947B04143009F444C01530F5
:1050300050F4113019F11130C0F0123051F1133029
:1050400009F074C02FC0173009F450C0183030F484
:105050001530D1F1163009F069C03FC0183009F49D
:105060004EC0193009F062C053C000D000D0EDB777
:10507000FEB7D283C18386E692E008C000D000D09C
:10508000EDB7FEB7D283C1838EE592E0948383832C
:1050900047C000D000D0EDB7FEB7D283C18386E50C
:1050A00092E0F4CF00D000D0EDB7FEB7D283C18339
:1050B0008EE492E0EBCF00D000D0EDB7FEB7D28304
:1050C000C183348223822CC000D000D0EDB7FEB75C
:1050D000D283C1835482438223C000D000D0EDB775
:1050E000FEB7D283C183748263821AC000D000D01D
:1050F000EDB7FEB7D283C1839482838211C000D002
:1051000000D0EDB7FEB7D283C183B482A38208C0BA
:1051100000D000D0EDB7FEB7D283C183D482C38262
:105120000E94372B0F900F900F900F908BE095E01F
:105130000E945F0461E070E080E090E00E9424340F
:105140000894E11CF11CF1EDEF16F7E0FF0609F001
:1051500058CFDF91CF911F91FF90EF90DF90CF90CC
:10516000BF90AF909F908F907F906F905F904F9087
:105170003F902F90089586E061E00E9401350895E8
:105180000F931F938091D105813009F051C00BE03E
:1051900015E0C8010E94C804C80163E04AE00E940B
:1051A000A303C8010E947B0400D000D0EDB7FEB776
:1051B000128301838EE692E0948383830E94372BCF
:1051C0000F900F900F900F90C8010E945F040E94F3
:1051D000290662E370E080E090E00E9424340E949F
:1051E000290662E370E080E090E00E9424340E948F
:1051F000290662E370E080E090E00E94243410927F
:10520000D10560ED77E080E090E00E942434C80191
:105210000E94C8041092FB020E9416340E94F536C8
:105220006093C6057093C7058093C8059093C90520
:105230000E9473258DE195E00E945A321F910F91D3
:1052400008950F931F93CF93DF9386E061E00E9450
:10525000C2340EEE14E0C80140E051EE60E070E0B0
:105260000E94592B10937806009377060E94BB2862
:10527000CBE0D5E0CE010E9401050E94D91764EF72
:1052800071E080E090E00E94243482EF93E00E947D
:1052900010088C34E1F0CE0163E049E00E94A303E2
:1052A000CE010E947B0400D000D0EDB7FEB7D283C0
:1052B000C18388E892E0948383830E94372B0F9008
:1052C0000F900F900F90CE010E945F04FFCF0E94BD
:1052D000A0071092780507C00E94561C809178059F
:1052E0008F5F80937805809178058230A8F31092C3
:1052F00078050E94C7278DE195E06AE07BE228E708
:1053000030E040E050E000E00E940C328BE095E09D
:105310000E94C8048DE195E00E947232DF91CF9126
:105320001F910F9108952F923F924F925F926F922B
:105330007F928F929F92AF92BF92CF92DF92EF9225
:10534000FF920F931F93DF93CF9300D000D0CDB780
:10535000DEB78091CA05882349F580915B058230CC
:1053600008F441C18091520590915305A0915405D4
:10537000B09155058093570690935806A09359060F
:10538000B0935A068091560590915705A091580503
:10539000B091590580935B0690935C06A0935D06DF
:1053A000B0935E0681E08093CA051DC1813009F08B
:1053B0001AC1A0905F0688E18A15B0F1E0907E05E1
:1053C000F0907F0500918005109181056091600645
:1053D000709161068091620690916306A801970121
:1053E0000E948E359F7720E030E040E05FE30E942E
:1053F0001F3818165CF410925F06E0926006F09277
:10540000610600936206109363060EC08A2D8F5FBB
:1054100080935F06893141F4E0928205F092830522
:105420000093840510938505E0905706F090580688
:105430000091590610915A06C801B7019F7725E3DC
:105440003AEF4EE85CE30E942A380E94593669839D
:105450007A838B839C83C801B701209152053091D8
:10546000530540915405509155050E948E351B01FE
:105470002C019F7720EC3BE649ED57E40E942A3847
:105480005B016C0160915B0670915C0680915D062A
:1054900090915E0620915605309157054091580530
:1054A000509159050E948E353B014C019F7720ECAD
:1054B0003BE649ED57E40E942A3829813A814B8125
:1054C0005C810E942A387B018C01C601B501A601CE
:1054D00095010E942A385B016C01C801B701A8013F
:1054E00097010E942A389B01AC01C601B5010E94B8
:1054F0008F350E94B1380E94C43660936005709366
:105500006105809362059093630560E070E080E838
:105510009FE329813A814B815C810E945C369B012B
:10552000AC01C201B1010E942A3897FA909497F811
:105530009094A40193010E94023620EE3EE245E6DB
:1055400052E40E942A3820E030E044EB52E40E940A
:105550008F350E94C4369B01AC0197FF04C02859C7
:105560003E4F4F4F5F4FCA01B901645B70408040AE
:10557000904097FF06C0CA01B9016C547F4F8F4F0E
:105580009F4F0E94F7362091400530914105409190
:105590004205509143050E948E350E94C43697FF04
:1055A00004C068597E4F8F4F9F4F0E94F73620E00E
:1055B00030E044EB53E40E945C3620E030E040E809
:1055C00051E40E942A380E948D3820E030E040E803
:1055D0005FE30E948F350E94C93660933A056131BE
:1055E00010F010923A050F900F900F900F90CF91FE
:1055F000DF911F910F91FF90EF90DF90CF90BF90C0
:10560000AF909F908F907F906F905F904F903F9062
:105610002F9008950E946F0A8BE095E00E949329D5
:105620000E94671908956EBD0DB407FEFDCF8EB5BB
:1056300008958DE061E00E94C2348BE061E00E9439
:10564000C2348CE060E00E94C2348AE061E00E94D3
:10565000C2341CBC80E58CBD8DB58EB5089584E642
:1056600096E00E94192B08958FEF9FE70895DF932E
:10567000CF93CDB7DEB7FE0139968D819E8161E073
:105680004F8158859F010E94D82DCF91DF910895B9
:10569000DF93CF93CDB7DEB7FE0139968D819E8122
:1056A00060E04F8158859F010E94D82DCF91DF91F6
:1056B00008950F931F93DC01ED91FC910288F3890B
:1056C000E02D20E030E000E010E009951F910F91FF
:1056D00008958F92AF92CF92EF92FF920F931F9304
:1056E000DF93CF93CDB7DEB7FC011382128288EE31
:1056F00093E0A0E0B0E084839583A683B78384E53C
:1057000094E0918380835587448737872687118B60
:10571000008BF38AE28AC48AA58A868A70E0CB016C
:1057200023E0880F991F2A95E1F79C012B59394FE7
:10573000308F278B8359994F928F818F81E090E032
:1057400002C0880F991F6A95E2F720917506282BF1
:1057500020937506CF0140E051EE60E070E00E94BA
:10576000592BCF91DF911F910F91FF90EF90CF9028
:10577000AF908F900895FC01838D882319F42FEF4B
:105780003FEF0DC00788F08DE02D208131818281AF
:105790009381281B390B8481958128233923C901E2
:1057A0000895FC01838D882319F42FEF3FEF11C07A
:1057B000018CF28DE02D2081318182819381281B23
:1057C000390B2095309584819581282339232F5FCB
:1057D0003F4FC9010895FC01838D882361F0A7899B
:1057E000B08D2D913C91119712968D919C911397AC
:1057F0002817390721F44FEF5FEFCA010895129679
:105800008D919C9113971696ED91FC911797E80F47
:10581000F91F408112968D919C91139701961496D1
:105820002D913C9115978223932313969C938E93ED
:10583000129750E0E2CFFC01838D882351F0078856
:10584000F08DE02D208131818281938128173907E5
:1058500021F42FEF3FEFC9010895828193810680E3
:10586000F781E02DE80FF91F8081282F30E0F3CF7A
:10587000DC015796ED91FC91589782819381918339
:1058800080835996ED91FC915A9780819181938301
:1058900082830895DC015B968C915B978823A9F144
:1058A0005996ED91FC915A97208131812F5F3F4F9E
:1058B00084819581282339235C968C915C97882379
:1058C00029F08281938128173907F9F08281938129
:1058D00028173907D9F3808191810680F781E02D5F
:1058E000E80FF91F60835996ED91FC915A97318327
:1058F00020835296ED91FC915397808156969C910E
:10590000892B808321E030E002C020E030E0C90133
:105910000895CF93DF93EC011B821A828A819B81C9
:10592000998388831D821C828E819F81009721F03C
:105930000E9436331F821E82DF91CF9108950F930C
:105940001F938C01DC015296ED91FC9153972081BD
:1059500056968C91569755969C915597892B809584
:105960008223808357968D919C9158970E94892C11
:10597000F801818D928D0E94892CD8015B961C9232
:105980001F910F9108950F931F93CF93DF938C0175
:10599000FC0113821282828193819183808341E092
:1059A000A1E0B0E001C04F5FFD01042E02C0EE0F88
:1059B000FF1F0A94E2F79B0182E06130780710F044
:1059C00020E032E0E217F30770F3C1E0D0E002C05C
:1059D000CC0FDD1F4A95E2F72197F8012681378128
:1059E0002115310541F0848195818C179D0789F03F
:1059F000C9010E943633F801D583C483CE010196D4
:105A00000E9499329C01F8019783868380E0232BC2
:105A100009F081E0DF91CF911F910F910895AF922E
:105A2000BF92CF92DF92EF92FF920F931F93CF938B
:105A3000DF937C015A016B01E901DC015B968C91DB
:105A40005B978823F1F02115310539F45796ED91D4
:105A5000FC915897C481D58121960115110549F40F
:105A6000D7015996ED91FC915A97048115810F5FEA
:105A70001F4FD701ED91FC910088F189E02DC701FE
:105A80000995F7018789908D209711F4C0E8D0E03F
:105A9000BE010E94C32C882381F0D70159968D91B5
:105AA0009C915A970115110511F400E110E0B8011D
:105AB0000E94C32C882309F04DC0D701ED91FC91C1
:105AC0000088F189E02DC701099567C0D70150967C
:105AD000ED91FC915197B0E0AB16B1EEBB06B0E092
:105AE000CB06B0E0DB0609F454C081E090E0D701BA
:105AF00054960C9002C0880F991F0A94E2F7808395
:105B000060E079E08DE390E0A60195010E9485397F
:105B10002150304040405040CA01B90122E030E0FD
:105B200040E050E00E948539D7011C96ED91FC9130
:105B30001D9730831E96ED91FC911F972083D7010E
:105B40005296ED91FC915397808155969C91892BAB
:105B5000808323C0D7015996ED91FC915A97138207
:105B6000128282819381918380835796ED91FC917B
:105B7000589713821282828193819183808381E07E
:105B80005B968C931A141B041C041D040CF49ECF0A
:105B9000D6CF108220E130E0C7CFDF91CF911F91A7
:105BA0000F91FF90EF90DF90CF90BF90AF9008954E
:105BB0002F923F924F925F926F927F928F929F921D
:105BC000AF92BF92CF92DF92EF92FF920F931F930B
:105BD000DF93CF93CDB7DEB764970FB6F894DEBFEF
:105BE0000FBECDBF3C01688B5A8B498B69011C01EC
:105BF000AE014F5F5F4F5C8B4B8BE989FA89488917
:105C000040FD659140FF6191FA8BE98B662309F4B1
:105C1000D7C3653249F440FD859140FF8191FA8BED
:105C2000E98B8532B1F40CC06A3051F4D301ED91A7
:105C3000FC910190F081E02DC1016DE009956AE0D1
:105C4000D301ED91FC910190F081E02DC101099506
:105C5000D4CF982F10E0882499241032B0F49B32CE
:105C600069F09C3228F4903251F0933271F40BC0F9
:105C70009D3239F0903349F4116028C012601460ED
:105C800025C0186023C0106121C017FD2BC0892FCB
:105C900080538A3078F416FF06C0BAE09B9E902CA1
:105CA0001124980E13C0EAE08E9E802C1124880ED9
:105CB00010620CC09E3221F416FD82C3106406C02F
:105CC0009C3611F4106802C0983661F4E989FA89AB
:105CD000488940FD959140FF9191FA8BE98B99237A
:105CE00009F0BBCF892F8554833020F4812F806148
:105CF000905E07C0892F8556833008F0E6C1812F5A
:105D00008F7E86FD02C076E0972E6FE3F62EF82296
:105D1000953619F450E4F52A07C0963619F480E850
:105D2000F82A02C091109A94F7FE0BC09BE39915D4
:105D300020F427E05CE3B52E0DC0B92CB39427E026
:105D400009C0A7E0A91520F447E0942E27E001C080
:105D5000292DBB24F6013496FD87EC87D6016D9181
:105D60007D918D919C91AE014F5F5F4F0B2D0E94F5
:105D700038026C010981E02FF0E0FF87EE8700FF19
:105D800005C0FE85F3FD02C01DE209C0F1FE02C0A0
:105D90001BE205C0F2FC02C010E001C010E28E85DB
:105DA0009F858C709070892B09F444C0112311F4E5
:105DB00083E001C084E0881510F088240EC0881AA2
:105DC000F3FC0BC0D301ED91FC910190F081E02D2B
:105DD000C10160E209958A94A9F7112349F0D30122
:105DE000ED91FC910190F081E02DC101612F0995A9
:105DF000BE85B3FF03C005EB13E012C009EB13E04F
:105E00000FC0E114F10409F06052D301ED91FC914F
:105E10000190F081E02DC10109950F5F1F4F05C072
:105E2000EF2CFF24B0E1EB22FF24F80164916623FC
:105E300041F748C1F7FE13C0BC0CFE85F4FF04C057
:105E40008A81813309F4BA941B141CF0BB24B394E7
:105E50002DC048E04B1550F538E0B32E27C0F6FCB6
:105E600025C0892D90E08C159D054CF05CEFC51682
:105E70005FEFD50624F080E8F82A01C09A949920B3
:105E800049F0E2E0F0E0EC0FFD1FE90DF11D80812B
:105E90008033A1F3F7FE0AC0B92CB394892D90E0AA
:105EA000C816D90614F0992401C09C18F7FC03C049
:105EB00025E030E009C01C141D041CF021E030E096
:105EC00003C096012F5F3F4F112311F02F5F3F4F0B
:105ED000992029F0892D90E00196280F391F882DEF
:105EE00090E02817390714F0882401C0821A4F2C3B
:105EF0005524C20189709070892B59F00CC0D301D0
:105F0000ED91FC910190F081E02DC10160E20995D5
:105F10008A948820A1F7112349F0D301ED91FC91D7
:105F20000190F081E02DC101612F099543FE0BC066
:105F30000CC0D301ED91FC910190F081E02DC101E5
:105F400060E309958A948820A1F7F7FE51C0860185
:105F5000D7FE02C000E010E076010894E11CF11CBD
:105F6000E01AF10AE1E0F0E0EC0FFD1FEE0EFF1E7B
:105F700026014B185108892D90E0AA24BB24A81AA9
:105F8000B90AFFEF0F3F1F0749F4D301ED91FC91D0
:105F90000190F081E02DC1016EE20995C016D10695
:105FA00034F0401651061CF4F701608101C060E333
:105FB000015010400894E11CF11C0A151B054CF01F
:105FC000D301ED91FC910190F081E02DC101099583
:105FD000D8CF0C151D0541F48A81863320F4853312
:105FE00019F4BE85B4FF61E3D301ED91FC9165C066
:105FF0006A81613309F00F7ED301ED91FC9101902C
:10600000F081E02DC10109959920E1F0D301ED91D6
:10601000FC910190F081E02DC1016EE2099512E042
:10602000E1E0F0E0EC0FFD1FE10FF11D60811F5F6B
:10603000D301ED91FC910190F081E02DC101099512
:106040009A9471F7D301ED91FC910190F081E02DCC
:1060500044FC02C065E601C065E4C1010995D7FCB6
:1060600005C0C114D10441F404FF06C0D094C1940A
:10607000D108D3946DE201C06BE2D301ED91FC91A4
:106080000190F081E02DC101099560E305C06F5FCB
:10609000E6EFFFEFCE0EDF1EFAE0CF16D104BCF71D
:1060A000D301ED91FC910190F081E02DC1010995A2
:1060B000D301ED91FC916C2D605D0190F081E02D9C
:1060C000C1010995CC84DD8478C1933631F09337D2
:1060D00099F0933509F061C023C0F601808189836E
:1060E0005E010894A11CB11C42E050E0C40ED51E14
:1060F00021E0E22EF12C12C0D601AD90BC9016FD2D
:1061000003C06FEF7FEF02C0692D70E0E2E0F0E0C6
:10611000CE0EDF1EC5010E9479037C011F7713C0DC
:10612000D601AD90BC9016FD03C06FEF7FEF02C0AB
:10613000692D70E0E2E0F0E0CE0EDF1EC5010E94A6
:106140006E037C01106813FF0BC023C0D301ED91D7
:10615000FC910190F081E02DC10160E209958A94E3
:10616000882D90E0E816F90688F313C0F50117FDB5
:10617000659117FF61915F01D301ED91FC91019051
:10618000F081E02DC101099581108A940894E108FD
:10619000F108E114F10451F710C1943611F0993669
:1061A00099F517FF0AC0F6012081318142815381A0
:1061B00084E090E0C80ED91E0CC0D6018D919C9150
:1061C0009C01442737FD4095542FE2E0F0E0CE0ECD
:1061D000DF1E9FE6F92EF12257FF09C0509540952A
:1061E000309521953F4F4F4F5F4FF0E8FF2ACA018E
:1061F000B901AE014F5F5F4F2AE030E00E9410030B
:10620000E82E4B89E41A41C0953721F41F7E2AE01D
:1062100030E01CC0197F9F3661F0903720F498352C
:1062200009F0CEC00FC0903739F0983709F0C8C0D8
:1062300004C028E030E00AC0106114FD146020E1C1
:1062400030E004C014FD166020E132E017FF08C002
:10625000D6016D917D918D919C91E4E0F0E008C0B4
:10626000D6018D919C91BC0180E090E0E2E0F0E0ED
:10627000CE0EDF1EAE014F5F5F4F0E941003E82E6F
:10628000FB89EF1A8FE7F82EF122F6FE0BC04EEFD6
:10629000F422E91438F4F4FE07C0F2FC05C05FEE06
:1062A000F52202C01E2D01C0192DF4FE0DC0FE0105
:1062B000EE0DF11D8081803319F489EEF82208C0BB
:1062C0001F5FF2FE05C003C08F2D867809F01F5FA7
:1062D0000F2DF3FC18C0F0FE13C0181510F09E2C03
:1062E0000FC09E2C980C911A182D0AC0D301ED9165
:1062F000FC910190F081E02DC10160E209951F5FE2
:106300001815A0F304C0181510F4811A01C08824D0
:1063100004FF17C0D301ED91FC910190F081E02DB5
:10632000C10160E3099502FF29C0D301ED91FC9101
:106330000190F081E02D01FD02C068E712C068E520
:1063400010C0802F8678D1F001FF02C06BE201C03F
:1063500060E2F7FC6DE2D301ED91FC910190F081D8
:10636000E02DC10109950AC0D301ED91FC91019086
:10637000F081E02DC10160E309959A94E914A0F33E
:10638000EA94D301ED91FC91A1E0B0E0AC0FBD1F08
:10639000AE0DB11D0190F081E02DC1016C91099508
:1063A000EE2071F70AC0D301ED91FC910190F081CC
:1063B000E02DC10160E209958A948820A1F71DCCE7
:1063C00064960FB6F894DEBF0FBECDBFCF91DF91BC
:1063D0001F910F91FF90EF90DF90CF90BF90AF9003
:1063E0009F908F907F906F905F904F903F902F90F5
:1063F0000895F999FECF72BD61BDF89A80B50895F0
:10640000F999FECF1FBA72BD61BD40BD0FB6F894B9
:10641000FA9AF99A0FBE08950F93FC016115710560
:1064200011F480E011C02183328343835483728747
:1064300061870170000F000F000F8081877F802B24
:1064400082608B7F808381E00F910895CF93DF93EB
:10645000EC010E9416349B01AC018D819E81AF81BD
:10646000B885281739074A075B0728F4888184FD17
:1064700002C060E00DC089819A81AB81BC81820F2E
:10648000931FA41FB51F8D839E83AF83B88761E0E0
:10649000222757FD2395332744275527922F9170A4
:1064A0009295907F88818F7E892B8883862FDF91BC
:1064B000CF910895CF93DF93EC01888182FF0FC0C5
:1064C000CE010E942632882351F0E985FA85309763
:1064D00009F00995888183FF02C08B7F8883DF9153
:1064E000CF910895CF93DF93EC0189859A85892B0D
:1064F000E1F089819A81AB81BC810097A105B1054A
:10650000A1F00E94163429813A814B815C81260FCB
:10651000371F481F591F2D833E834F83588788811B
:1065200084608F7E888381E001C080E0DF91CF911D
:1065300008950F931F93CF93DF93BC018230910591
:1065400010F462E070E0E0918606F091870640E08A
:1065500050E0A0E0B0E024C08081918186179707C9
:10656000D0F08617970771F482819381109729F0F4
:1065700013969C938E9312972CC0909387068093CA
:10658000860627C04115510519F08417950718F4A0
:106590008D01AC01EF01DF01828193819C01F90142
:1065A0003097D1F641155105F9F0CA01861B970BBA
:1065B0008430910580F48A819B810115110521F0B9
:1065C000F8019383828304C09093870680938606A4
:1065D000FE01329645C0FE01E80FF91F61937193E9
:1065E0000297998388833CC08091840690918506A8
:1065F000892B41F4809104039091050390938506C3
:10660000809384064091060350910703411551057C
:1066100041F44DB75EB78091020390910303481B8C
:10662000590B209184063091850624173507B0F464
:10663000CA01821B930B8617970780F0AB014E5F50
:106640005F4F8417950750F0420F531F50938506F4
:1066500040938406F9016193719302C0E0E0F0E099
:10666000CF01DF91CF911F910F910895CF93DF93C9
:106670009C01009709F48FC0EC0122971B821A82BB
:1066800060918606709187066115710581F4888195
:106690009981820F931F20918406309185062817D7
:1066A000390739F5D0938506C093840674C0DB01A1
:1066B00040E050E0AC17BD0708F1BB83AA83FE01A0
:1066C00021913191E20FF31FAE17BF0779F48D913D
:1066D0009C911197280F391F2E5F3F4F39832883D4
:1066E00012968D919C9113979B838A834115510536
:1066F00071F4D0938706C09386064DC012968D9193
:106700009C911397AD01009711F0DC01D3CFDA0112
:106710001396DC93CE931297FA0121913191E20FF7
:10672000F31FCE17DF0769F488819981280F391F7D
:106730002E5F3F4FFA01318320838A819B819383AF
:106740008283E0E0F0E0DB0112968D919C9113973B
:10675000009719F0BC01FD01F6CFAB014E5F5F4F12
:10676000DB018D919C91840F951F209184063091BF
:1067700085062817390779F4309729F4109287068F
:106780001092860602C013821282425050405093EB
:10679000850640938406DF91CF9108951F920F9252
:1067A0000FB60F9211242F933F938F939F93AF9324
:1067B000BF9380917F0690918006A0918106B09151
:1067C0008206309183060196A11DB11D232F2D5FF6
:1067D0002D3720F02D570196A11DB11D2093830662
:1067E00080937F0690938006A0938106B0938206E3
:1067F00080917B0690917C06A0917D06B0917E06EB
:106800000196A11DB11D80937B0690937C06A093F9
:106810007D06B0937E06BF91AF919F918F913F917E
:106820002F910F900FBE0F901F9018958FB7F8946F
:1068300020917F063091800640918106509182061A
:106840008FBFB901CA0108959B01AC017FB7F894CD
:1068500080917B0690917C06A0917D06B0917E068A
:1068600066B5A89B05C06F3F19F00196A11DB11D2B
:106870007FBFBA2FA92F982F8827860F911DA11DA2
:10688000B11D62E0880F991FAA1FBB1F6A95D1F73F
:10689000BC012DC0FFB7F89480917B0690917C06D7
:1068A000A0917D06B0917E06E6B5A89B05C0EF3F9E
:1068B00019F00196A11DB11DFFBFBA2FA92F982F66
:1068C00088278E0F911DA11DB11DE2E0880F991F31
:1068D000AA1FBB1FEA95D1F7861B970B885E9340D2
:1068E000C8F2215030404040504068517C4F211543
:1068F00031054105510571F60895019739F0880F6A
:10690000991F880F991F02970197F1F708957894BE
:1069100084B5826084BD84B5816084BD85B58260A4
:1069200085BD85B5816085BDEEE6F0E08081816042
:106930008083E1E8F0E01082808182608083808142
:1069400081608083E0E8F0E0808181608083E1EB1A
:10695000F0E0808184608083E0EBF0E08081816002
:106960008083EAE7F0E080818460808380818260B8
:1069700080838081816080838081806880831092A1
:10698000C1000895CF93DF93482F50E0CA01815191
:106990009C4FFC01349145525C4FFA01849188234D
:1069A00069F190E0880F991FFC01E354FC4FA59119
:1069B000B491FC01E953FC4FC591D491662351F485
:1069C0002FB7F8948C91932F909589238C9388817D
:1069D00089230BC0623061F42FB7F8948C91932F08
:1069E000909589238C938881832B88832FBF06C041
:1069F0009FB7F8948C91832B8C939FBFDF91CF919D
:106A00000895482F50E0CA018D5F9B4FFC012491EF
:106A1000CA0181519C4FFC01949145525C4FFA018F
:106A20003491332309F440C0222351F1233071F013
:106A3000243028F42130A1F0223011F514C0263082
:106A4000B1F02730C1F02430D9F404C08091800027
:106A50008F7703C0809180008F7D8093800010C06D
:106A600084B58F7702C084B58F7D84BD09C08091C5
:106A7000B0008F7703C08091B0008F7D8093B0000D
:106A8000E32FF0E0EE0FFF1FE953FC4FA591B49107
:106A90002FB7F894662321F48C919095892302C036
:106AA0008C91892B8C932FBF0895CF93DF930E94F5
:106AB00087340E942129C0E0D0E00E94C02820979E
:106AC000E1F30E940000F9CFCF92DF92EF92FF92A4
:106AD0000F931F93CF93DF937C016B018A01C0E07A
:106AE000D0E00FC0D6016D916D01D701ED91FC9101
:106AF0000190F081E02DC7010995C80FD91F015001
:106B000010400115110571F7CE01DF91CF911F9152
:106B10000F91FF90EF90DF90CF9008955058BB27D2
:106B2000AA270ED041C201D230F006D220F031F4B3
:106B30009F3F11F41EF4C0C10EF4E095E7FBB6C10F
:106B4000E92F54D280F3BA176207730784079507B9
:106B500018F071F49EF56CC20EF4E0950B2EBA2F6E
:106B6000A02D0B01B90190010C01CA01A001112453
:106B7000FF27591B99F0593F50F4503E68F11A16FF
:106B8000F040A22F232F342F4427585FF3CF469590
:106B900037952795A795F0405395C9F77EF41F16B2
:106BA000BA0B620B730B840BBAF09150A1F0FF0F7C
:106BB000BB1F661F771F881FC2F70EC0BA0F621F68
:106BC000731F841F48F4879577956795B795F79558
:106BD0009E3F08F0B3CF9395880F08F09927EE0FEA
:106BE000979587950895A1D158F080E891E009F430
:106BF0009EEFA2D128F040E851E059F45EEF09C0C1
:106C00005BC116C2E92FE078F1D168F3092E052A9D
:106C1000C1F3261737074807590738F00E2E07F833
:106C2000E02569F0E025E0640AC0EF6307F800940E
:106C300007FADB01B9019D01DC01CA01AD01EF9347
:106C40004AD0B2D10AD05F91552331F02BED3FE00D
:106C500049E450FD49EC63CF0895DF93DD27B92F58
:106C6000BF7740E85FE31616170648075B0710F486
:106C7000D92FE9D19F938F937F936F93BCD2EAE88A
:106C8000F0E01DD191D12F913F914F915F91EED1C5
:106C9000DD2349F09058A2EA2AED3FE049EC5FE39A
:106CA000D0785D274DDFDF917FC1DCD008F481E033
:106CB00008954AD1E39589C10CD076C13DD140F009
:106CC00034D130F021F45F3F19F0F0C05111B1C15F
:106CD000F3C08CD198F39923C9F35523B1F3951BD5
:106CE000550BBB27AA2762177307840738F09F5FED
:106CF0005F4F220F331F441FAA1FA9F333D00E2E5C
:106D00003AF0E0E830D091505040E695001CCAF7C8
:106D100029D0FE2F27D0660F771F881FBB1F26178D
:106D200037074807AB07B0E809F0BB0B802DBF0160
:106D3000FF2793585F4F2AF09E3F510568F0B6C079
:106D400078C15F3FECF3983EDCF3869577956795C5
:106D5000B795F7959F5FC9F7880F911D9695879511
:106D600097F90895E1E0660F771F881FBB1F621730
:106D700073078407BA0720F0621B730B840BBA0BEE
:106D8000EE1F88F7E095089504D06894B11151C1C1
:106D9000089534D188F09F5790F0B92F9927B751B3
:106DA000A0F0D1F0660F771F881F991F1AF0BA95CF
:106DB000C9F712C0B13081F03BD1B1E0089538C1BC
:106DC000672F782F8827B85F39F0B93FCCF38695C5
:106DD00077956795B395D9F73EF490958095709522
:106DE00061957F4F8F4F9F4F0895E89409C097FB9F
:106DF0003EF490958095709561957F4F8F4F9F4F92
:106E00009923A9F0F92F96E9BB279395F6958795D5
:106E100077956795B795F111F8CFFAF4BB0F11F498
:106E200060FF1BC06F5F7F4F8F4F9F4F16C088233F
:106E300011F096E911C0772321F09EE8872F762F75
:106E400005C0662371F096E8862F70E060E02AF0B6
:106E50009A95660F771F881FDAF7880F96958795A2
:106E600097F90895990F0008550FAA0BE0E8FEEF77
:106E700016161706E807F907C0F012161306E407FE
:106E8000F50798F0621B730B840B950B39F40A26F7
:106E900061F0232B242B252B21F408950A2609F4D5
:106EA000A140A6958FEF811D811D089597F99F67D9
:106EB00080E870E060E008959FEF80EC0895DF9334
:106EC000CF931F930F93FF92EF92DF927B018C0180
:106ED000689405C0DA2EEF01C9D0FE01E894A591AF
:106EE0002591359145915591AEF3EF0129DEFE01D3
:106EF0009701A801DA9479F7DF90EF90FF900F9156
:106F00001F91CF91DF9108959F938F937F936F93FC
:106F1000FF93EF939B01AC019DD0EF91FF91CFDFE9
:106F20002F913F914F915F9195C000240A941616BE
:106F3000170618060906089500240A941216130667
:106F4000140605060895B8CF59D0E8F3E894EFEF9A
:106F5000BB273FE048EC5FE76B3D7307840795076D
:106F600008F1FF279F57B25A6A4D7F40894CF04085
:106F700032F4BE556542704F8643FF4F0894EE1FB2
:106F8000915030F0BB0F661F771F881FFF1FEBCF9C
:106F90009EE7882332F0BB0F661F771F881F9A95E4
:106FA000C1F79395E09565C1092E0394000C11F487
:106FB000882352F0BB0F40F4BF2B11F460FF04C0D4
:106FC0006F5F7F4F8F4F9F4F0895EF93E0FF06C095
:106FD000A2EA2AED3FE049EC5FEBB2DDE5DF0F907E
:106FE000039401FC9058E7EBF0E08ECF57FD9058EA
:106FF000440F551F59F05F3F71F04795880F97FB7D
:10700000991F61F09F3F79F0879508951216130636
:107010001406551FF2CF4695F1DF08C01616170665
:107020001806991FF1CF869571056105089408959A
:10703000E894BB2766277727CB0197F9089512DFDD
:1070400008F48FEF08959B01AC0160E070E080E8E8
:107050009FE332CE0BD0A8CF68DF28F06DDF18F0A9
:10706000952309F023CF28CF1124E3CFBFDFA0F36E
:10707000959FD1F3950F50E0551F629FF001729FCD
:10708000BB27F00DB11D639FAA27F00DB11DAA1FEC
:10709000649F6627B00DA11D661F829F2227B00D39
:1070A000A11D621F739FB00DA11D621F839FA00DC4
:1070B000611D221F749F3327A00D611D231F849F14
:1070C000600D211D822F762F6A2F11249F5750406B
:1070D0008AF0E1F088234AF0EE0FFF1FBB1F661F06
:1070E000771F881F91505040A9F79E3F510570F0BF
:1070F000DDCE9FCF5F3FECF3983EDCF3869577952E
:107100006795B795F795E7959F5FC1F7FE2B880FB9
:10711000911D9695879597F9089570DFE0F09E3759
:10712000D8F09639B8F49E3848F4672F782F88271E
:10713000985FF9CF86957795679593959539D0F3B4
:10714000B62FB1706B0F711D811D20F48795779557
:107150006795939573C08DC06CCF11F40EF4ACCECF
:1071600088C04CDFD0F39923D9F3CEF39F57550B4A
:1071700087FF8FD056959795B0E020F4660F771F64
:10718000881FBB1F1F930F9300249001A001800153
:10719000F001A0E80E0F1F1F0A1E511D601B710B8E
:1071A0008009B50B48F4600F711F801DB51F0E1BC1
:1071B0001F0B0A0A510907C02E0F3F1F4A1F0E0F4F
:1071C0001F1F0A1E511D660F771F881FBB1FA69524
:1071D000F795E795F8F60617170708065B07211DD0
:1071E000311D411D0F911F91B901842F9158880FB6
:1071F0009695879508959B01AC012CCFDF93D92FED
:10720000A3DEE695D7952AED3FE049E45FE3B33A84
:107210006207730784079507D7952AF0A2EA49EC1D
:1072200090688EDCC1DEE5EDF0E06EDEDD0F0BF088
:107230000ADFDD0F0BF49058DF910895882371F475
:10724000772321F09850872B762F07C0662311F4FF
:1072500099270DC09051862B70E060E02AF09A9536
:10726000660F771F881FDAF7880F9695879597F92D
:1072700008959F3F49F0915028F48695779567953A
:10728000B7959F5F80389F4F880F9695879597F9A0
:10729000089591505040660F771F881FD2F70895C8
:1072A00097FB092E07260AD077FD04D049D006D0D7
:1072B00000201AF4709561957F4F0895F6F7909528
:1072C00081959F4F0895A1E21A2EAA1BBB1BFD01B9
:1072D0000DC0AA1FBB1FEE1FFF1FA217B307E407B5
:1072E000F50720F0A21BB30BE40BF50B661F771F0D
:1072F000881F991F1A9469F76095709580959095ED
:107300009B01AC01BD01CF01089597FB092E052615
:107310000ED057FD04D0D7DF0AD0001C38F45095AA
:107320004095309521953F4F4F4F5F4F0895F6F7A9
:1073300090958095709561957F4F8F4F9F4F0895E1
:10734000AA1BBB1B51E107C0AA1FBB1FA617B7078B
:1073500010F0A61BB70B881F991F5A95A9F78095A7
:107360009095BC01CD010895EE0FFF1F0590F4919B
:08737000E02D0994F894FFCF11
:10737800256300256325332E306625637C25632528
:1073880063002563256300007374616200616372A2
:107398006F00616C7468006175746F00677569646B
:1073A800006C6F6974007265746C006369726300C5
:1073B800706F7369006C616E64006F666C6F006457
:1073C800726966007370727400666C69700061742B
:1073D800756E0068796272006D616E750074726E08
:1073E800670066627761006662776200637275693A
:1073F80000696E6974002563257300256325326969
:10740800256325342E306625630025737C25632586
:107418007325630020C0C0C0C0C0C7C0C0C0C0C002
:10742800200025342E306625630025632531312E52
:1074380036667C25632531312E3666002563253274
:107448006900102000112000257300256325352EC2
:107458003266256300253469256325630025632585
:10746800352E3066256300256325332E3069256364
:1074780000256325332E30662563002563256325A3
:10748800322E306625637C2563256325322E3066CF
:1074980025637C2563256325342E306925637C2587
:1074A80063256325342E306925637C256325632590
:1074B800332E306625637C2563256325332E30669D
:1074C80025637C2563256325342E306625630025D6
:1074D80063253369256300256325326925632530D3
:1074E800326900256325342E306625630020204448
:1074F800495341524D45442020002020202020207F
:1075080020202020202000204E6F20475053206646
:10751800697821002020205374616C6C2120202080
:1075280000204F76657253706565642120004261C2
:107538007474657279204C6F77210020204C6F7726
:10754800205273736920200025332E30692563008B
:1075580025332E3166256300000080BF000080BF00
:107568009DFF64E803E803E803E803010C01000059
:10757800000080008806000000000000AB046435AD
:10758800A903AC03AF03B203342B327C8900EDD9D5
:107598006877000000590000000000000000D69F36
:1075A800DCA81817AA90437327F6B968EDF4DED45F
:1075B80009FEE61C1C84DDE80B992927D6DF8D21FE
:1075C8000F036418EFEE1EF0B782820094150034A2
:1075D8007C0000001400988F0000000000000000EC
:1075E800000000E7B73F3600000000000000AF666B
:1075F8009ED03800000000000000000000000000DD
:107608000000000000000000000000000000000072
:107618000000000000000000000000000000000062
:1076280086DBD0BC5416131586004E44BD7F6F15FB
:10763800159001000000000000000000000000009C
:107648000000000000000000000000000000000032
:107658000000000000000000000000000000000022
:107668000000000000000000000000000000000012
:107678000000000000000000000000000000000002
:10768800000000CC31AA2C532E0002000200050095
:10769800020005000200010203060A0BC2C0C0C1B5
:1076A800C0C0C1C0C0C4C0C0C1C0C0C1C0C0C3C0C8
:1076B800C0C1C0C0C1C0C0C5C0C0C1C0C0C1C0C0B9
:1076C800000000004A2C6435BB2BEB2B1B2C382CFC
:0876D800D12B592B9F2C0F2D23
:00000001FF
